:020000040000fa
:080000000002040000000000f2
:020000040000fa
:10040000ef4421000e7f22000e0188000000000052
:100410000c000700e01b2300010020001100070072
:10042000000020000000e000020032000000020096
:1004300000000000b0420200000000000040da00ae
:100440000000fe004440a900406820000000e000d9
:100450000300320000002000a00188004440a800f2
:100460000000060091018800800078000000eb0089
:1004700015003700e280400032a0b4009101ba00bc
:10048000e280400032a0b4009102ba00e280400055
:1004900032a0b4000002eb00472bde00f507b200eb
:1004a000602ce10004003a000059eb008301e900f0
:1004b000fdff3e00040037006128e100010032002a
:1004c0000082eb00040007001101ba000200e00006
:1004d000e8ff3a00000006003159ba008301e90044
:1004e0000c0032002159ba008301e90008003200f3
:1004f0000400e00003003a00e280400032a0b400b3
:10050000f5ff370011d9ba008301e900faff3a007c
:100510008100e800e180400032a0b4000000060045
:1005200000000000000000000000000000000000cb
:1005300000000000000000000000000000000000bb
:1005400000000000000000000000000000000000ab
:10055000000000000000000000000000000000009b
:10056000000000000000000000000000000000008b
:10057000000000000000000000000000000000007b
:10058000000000000000000000000000000000006b
:10059000000000000000000000000000000000005b
:1005a000000000000000000000000000000000004b
:1005b00000000000000000000040da000000fe0023
:1005c000800078001106b100030035009101b100f0
:1005d00001003c000050a100000006000003b10033
:1005e0000b0035009000b100080034008000b1001d
:1005f000070035009001b100040034007000b10024
:10060000030035009001b10001003c00100005001e
:10061000000005000a00fa0080017800e20f500097
:1006200028003e0060a28000e10f50000800320068
:10063000802320000000e000050032000423200099
:100640002523200046232000800178000400370085
:1006500004222000252220004622200083222000a0
:10066000144090000004e000040035008009eb0015
:10067000144090000074a0001042980015409000b3
:100680000028a30003003a00154090000024a000b9
:10069000904298008001eb00070037001540900061
:1006a0000008a300fdff320063c078000000fb00db
:1006b000000b78008301e800828f5100f7ff3a00b9
:1006c0000800370030002000b0bf9f00c3bf9f006c
:1006d000d1bf9f00e2bf9f006a80570000c0da00d0
:1006e0006fb99700020078000080fa000000060051
:1006f0000001be00200107000470a70003f0a10064
:100700006509b100160032000d0035006828e100cf
:1007100006003500f0ff2f00f1ff27000300e00086
:1007200013003b000100280000000500000040000d
:10073000818048008502e900fcff3a00080037008c
:10074000f88f420002003c008000eb000000050032
:100750008100d1000080d3008502e800fcff3a0050
:100760000300e00002003b0060001000e080180081
:1007700000000600889fbe008a9fbe000105780029
:100780000100e0000400350008003c000000e0002b
:10079000200032000500370060001000e0801800e3
:1007a00002003b0001f02c001a0037000004be00dc
:1007b0006011b8006b0920000982cf0002003900e7
:1007c0000882cf000441b000694252000e0032009e
:1007d00008003b0082817100610164008904d1003e
:1007e0000884d3008b05e8000442e800f9ff3a00d2
:1007f000050037000804440089844c008b05e9009b
:100800000442e900fbff3a00f00007000af0a700ed
:1008100001f0a0004f05be004f04be00000006001e
:1008200003f0a200889fbe008a9fbe008c1f780044
:100830000c010700130133006450e1004f00320047
:100840006420e1005200320003826c0007003b008c
:100850000905d0000306d000820f54000c065d008d
:100860000200390002003200890178000306780096
:100870008582550004003d000003fd008103fd005a
:100880008502ea008b854200840f720002003b0063
:1008900060001000e08018006011b8000005eb0057
:1008a0007a28e1000a00390006007800c75ddd0003
:1008b000f707b200878075002d0037008281710034
:1008c0000a017800610560008180d1000080d300ba
:1008d0008502e900f9ff3b000604400087844800d8
:1008e00002003b0060041400e0841c000988a3009f
:1008f000070032008a817100828171006101640009
:100900008904d1000884d3008b05e8001700370064
:100910000978a30013003a000b00e0001300340034
:100920008b05e9000804440089844c000a447400e3
:100930000978a3000d003a000b00e0000700340026
:100940008b05e9000804440089844c0001003a004a
:100950000b0020000978a300f7ff32000001eb0034
:1009600002003700828171000a01780097000700b9
:100970000cf0a70001f0a000cb0037006420e100dc
:1009800002003a00838f6c00cb0033000801be00e8
:100990000200be00c4003700889fbe008a9fbe00d0
:1009a0008c1f7800af000700b600330003866c0090
:1009b0006450e100240032006420e100270032008e
:1009c0006150e100220032006120e100210032008c
:1009d0008b854200eb07b1000134b800003ab80043
:1009e0000804420089844a00013ab8000030b80087
:1009f0008880400009014a000400330000004000e4
:100a000081804800020149008b05e900c909dd0029
:100a1000830170000100320013002000c814de00c2
:100a20004814dd004709de001200b200c808de00ed
:100a3000088470006500070001f0a1000cf0a70019
:100a400001f0a000980037006120e1009a00320018
:100a50000801be000200be00f7ff37006150e10050
:100a6000fcff3a0094003700889fbe008a9fbe00ba
:100a70008c1f78007b0007008200330003866c0027
:100a80006450e1002e0032006420e10033003200a7
:100a90006150e1002f0032006120e100310032009e
:100aa00085855500eb07b0000900200008042000f0
:100ab000050037000804440089844c000a00310016
:100ac0000603430087834b000001530081815b00d4
:100ad000f8ff33000203be000800a0000804440031
:100ae00089844c00f6ff3900c639dd0083017300ac
:100af00001003200130020008904d1000884d300d3
:100b00000998a300050032000800a7000300a00018
:100b10008904d1000884d3008b05e8008904d10042
:100b20000884d3000001eb000281d20027000700f7
:100b300001f0a1000cf0a70001f0a0005a0037005e
:100b40006420e1005c0032000801be000200be002b
:100b5000f7ff37006120e100570032006000b80065
:100b6000f3ff37000000200001f82700f0ff3700f6
:100b70001400200053003700c70ade00f107b2005e
:100b8000f50fb20008003200e1cf4200020032004f
:100b90000170a00024000500810f700001003200e8
:100ba0000408050044000500810f700002003a00af
:100bb000140005008502e9000000400081c04800e3
:100bc000fcff3b000170a000240005008100200014
:100bd000618055000b003d000b00200061fe2f00de
:100be0000100e1001d003400828171006101640098
:100bf0008904d1000884d3000000e800faff3a001d
:100c000071002000610064000300700002006000b9
:100c10000900320061044400e0844c000988a5000a
:100c2000050032008b05e8006808e10002003a0088
:100c30008904d1000884d300f20f20000258e1009b
:100c400005003d00c75ddd00f907b2008980750031
:100c500008007800000006000bf827008b007800e1
:100c6000000005000004be00c3ff07000003be0033
:100c70000405be000200be00bfff0700844f7500e0
:100c8000000006000200be006450e10005003600ce
:100c90006420e100020036000968a30001003a0068
:100ca0000800be000160a0004f0678004f05be009e
:100cb0004f04be0000000600f0ff2f00f1ff2700e8
:100cc000f9ff3700889fbe008a9fbe00841f78000e
:100cd000e4ff07004f00780011003300f0ff2f0001
:100ce000838f6c0006003b00040565000a00a70026
:100cf0000800370009f0a6001000200008003700a7
:100d0000820f5400838f5c00030039001000200024
:100d100001003e000000200009f0a7000000ea00ea
:100d20004f05be004f04be000000e00000000600ba
:100d3000881f7800000478005001be004000be000b
:100d40000400400085804800060149008781490071
:100d5000009cbe000294be000400e1000588e10092
:100d60000690e1000798e1000200310068004400ad
:100d70001008e8004f04780000000600f4874700e0
:100d8000889fbe008a9fbe008c9fbe008e1f780089
:100d90000205be000004be00d4b79f00e5b79f0067
:100da000f6b79f0087bf9f000000eb00c0b79f0011
:100db000b0b79f00a0b79f0090b79f0080b79f007b
:100dc0000d042000bfb097004fb097000001400015
:100dd0000000e0000f003d004f08de000000710041
:100de000c0b79f009e00070001003d0012002000d8
:100df000a100070001003d0012002000a60007002e
:100e0000b1000700b60007000f004000c8ff070050
:100e1000220037004f08de0000067100ccb79f00ab
:100e20008f00070001003d00120020009200070023
:100e300001003d001200200097000700a2000700fb
:100e40000fb297009fb297002fb39700bfb39700e0
:100e5000a90007000000520081805a0002015b00d7
:100e600083815b0080b79f0091b79f00a2b79f006e
:100e7000b3b79f000007eb009f0007000020e100d0
:100e800001a8e10002b0e10003b8e1000100310077
:100e90001e0020000e005600c0b79f004fb2970002
:100ea0000400e000070035001000200001002000d1
:100eb0006011b80008047000898470000a05710090
:100ec0008b8571008d06e900beff3a000400e0004a
:100ed00003003d00820007000f00400094ff070060
:100ee0004fa897000000e00004003a000fb49700fc
:100ef0009fb497002fb59700bfb5970094000700e7
:100f00004f0778004f06be004f05be004f04be00dd
:100f10004f01b10000000600881f78001800200073
:100f2000881f780095ff07008f87e9004f0478003d
:100f300000000600801feb0090ff07008f87e9008c
:100f400000000600889fbe008a9fbe008c1f7800ac
:100f50006e00070007003d0073000700e00f5b0014
:100f6000e08f5b0007003d00320007000006eb0049
:100f7000040037003400070002003d002a0007008b
:100f80001c00200072000700e3ff07000203be0000
:100f90000002be000c00e000010032002200070049
:100fa0000400be000601be004f0678004f05be00db
:100fb0004f04be0000000600889fbe008a9fbe004e
:100fc0008c1f78005100070005003d005600070007
:100fd000e00f5b00e08f5b0006003d00040037007f
:100fe0001900070003003d006000b8006011b80060
:100ff0001000070056000700ceff07000203be00e6
:101000000002be000c00e0000100320006000700f4
:101010000400be000601be004f0678004f05be006a
:101020004f04be00000006006000b8006011b80068
:101030000000370004025000858258000603590062
:1010400087835900000006000006eb00e00f520005
:10105000e08f5a00e00f5b00e08f5b0000000600ad
:101060000180400090b79f000001eb008fb0970017
:101070000100e000000006000200700090b79f0031
:101080000180400080b79f000001eb00ffa897009f
:101090000100e000000006000200700080b79f0021
:1010a000018040006faa9700cf20de000100700091
:1010b000f0af9f0004024200250007004f18de0039
:1010c0000002720000000600e4af9f000804440024
:1010d00089844c000a054d008b854d0000000600f8
:1010e0003fb29700cfb297005fb39700efb397007e
:1010f00000fe2f00000006003fb09700cfb0970021
:101100005fb19700efb19700000006000205be0036
:101110000004be00e00f5000e08f5800e00f5900bf
:10112000e08f5900000006006000b8006011b800b0
:1011300008045000898458000a0559008b8559001d
:101140001c002000e00f5200e08f5a000000060053
:101150000800be000a01be00000006002800fa00d8
:10116000889fbe008a9fbe008c9fbe0003866b00d6
:101170000c0207000028a30064003a000128a30025
:1011800067003a000008a30062003a000108a300cb
:1011900065003a001e009000be08900081064000e5
:1011a000ed3fb100f4805700ee019000111ab80035
:1011b0008e099000311bb8009e099000311cb800c8
:1011c000511db800f485570046000700fe0190004d
:1011d0003a0007008b85e8003e0007008e0990006a
:1011e00040000700ee019000340007008b85e80006
:1011f000380007008e099000400007009e0990000b
:101200001b18b800890440000a854800fe019000c0
:10121000340007008b85e80038000700ee019000dd
:10122000300007008e0990001b18b80089044000a8
:101230000a8548000a98a30008003a000402420008
:1012400085824a0006034b0087834b0008044c004c
:1012500089844c000a054d008d06e90084827200e5
:10126000850273004c3add008502720001003200f5
:1012700015002000443ade001400b2004538de00bc
:10128000cb45dd000b007000c540de00cb4ddd001e
:101290008b8070004549de00cb55dd000b017100ed
:1012a000c551de000d037800d701070003f0a1004f
:1012b0000cf0a70003f0a000ce0137001b18b80007
:1012c0008502400006834800e0834b0060044c0028
:1012d000070037001b18b80006034000878348004a
:1012e000faff37001b18b800870340000884480045
:1012f000e0844c0060054d00000006001b18b8009b
:101300000804400089844800faff37000108a30060
:10131000b5013a005800be005801be00e3ff370097
:101320000008a300b0013a0009047800f9ff370073
:101330008103780010fe07000001be006000b800c5
:101340000478a30013003a006220e10015003e007b
:101350000d0039008301d1000281d3008180d300c8
:101360008301d1000281d3008180d3008301d100a9
:101370000281d3008180d3000538b000c42add008b
:10138000f300b2008381720007f0a70003f0a00011
:1013900000000600f3ff2700f2ff2f006110b900e4
:1013a000fbff370003ff2700f7ff37008f1fd10037
:1013b000c10107008f87e9000000e000000006007f
:1013c000801feb00bc0107008f87e9000000e000f0
:1013d000000006001400fa00889fbe008a9fbe002d
:1013e0008c9fbe000005be000206be0068004700dc
:1013f0000c90be000a90be00d80107006400e10016
:101400001a00320016003e006100e1001a003200ae
:101410006e049000fe0490000e0b90009e0b900056
:101420006011b8009e0590000b38b100d501200076
:1014300082817100610164008703d1000683d300bb
:101440008984d3000884d3008502e900f8ff3a00bc
:10145000defd07000df0a70001f0a00065013700d8
:10146000f1ff2700f0ff2f006201370001f827008d
:1014700000002000f7ff37006000b800f5ff3700dc
:10148000dd0107000509780000000600809feb00e1
:10149000890107008f87e9000000e00000000600d6
:1014a0002800fa00889fbe008a9fbe008c9fbe0065
:1014b00007067800878669000c003b00030478006b
:1014c0008704780008f0a10009f0a100840f500003
:1014d000858f5800860f5900890f5c000300330088
:1014e0000cf0a20001003a000cf0a1002d01070051
:1014f0006400e1005f003200780147006408e10009
:10150000610032006c014700748557003200be0054
:101510001201be003a04be001a05be001e03900070
:10152000be0a90008503530006003d000004fd0044
:101530008104fd000205fd008305fd008703ea002c
:10154000050378000df8a3000400320060041400c5
:10155000e0841c0060051d00e0851d006022b800cd
:101560007d0320000d38e1008006eb000b00390000
:101570004433dd00f300b20083017300390037000b
:10158000848272000d027800e10664008b85d10030
:101590000a85d3008984d3000884d3008703e90037
:1015a000f7ff3b0008004000898048000a0149001d
:1015b0008b81490004003b0060001000e0801800af
:1015c00060011900e08119000358a30009003200ee
:1015d0008d82720084827200610260008301d100fa
:1015e0000281d3008180d3000080d3000603e8008d
:1015f0001b0037000348a30017003a000600e00074
:10160000170034000603e9000d00a30000004800a5
:101610008180480002014900838149000348a300fa
:101620000f003a000600e000090034000603e9005c
:101630000000400081804800020149008381490088
:1016400001003a000003eb000348a300f5ff32005d
:101650006022b80002003700848272006182660056
:10166000e900070003f0a1000cf0a70003f0a000c0
:10167000e0003700640147006408e10002003a001e
:101680000df8a300d8003a003200be001201be00df
:10169000d80037001400fa00889fbe008a9fbe0061
:1016a0008c9fbe000004be000205be00680047001b
:1016b0000a90be000890be00280107000070a70035
:1016c0000bf0a1000bf8a30020003a009e09900047
:1016d0000e099000fe0090006e0090009e029000a7
:1016e0003443200084825200c20032000a003c00d1
:1016f000b4fc2f000428e100140034008301d10061
:101700000281d3008180d3000080d3008502e800ed
:10171000faff3a00b7003700b40020000428e100c7
:1017200007003c00000040008180480002014900a1
:10173000838149008502e900faff3a00ad003700d5
:101740000300280002002000010037006011b800eb
:101750006000b800a70037002800fa00889fbe008c
:101760008a9fbe008c9fbe0003866b008d00070021
:101770006400e100440032006408e1004a003200e5
:101780006100e100460032006108e10049003200da
:10179000ec0647006000b8003d02be003d03be00fd
:1017a000f48657006011b8003d04be003d05be0040
:1017b0007d0320000b0037000000a0008d06e9002b
:1017c000130032000402420085824a0006034b00e7
:1017d00087834b00000040008180480002014900df
:1017e000838149000802520089825a000a035b0083
:1017f0008b835b00f0ff3b000802420089824a00b5
:101800000a034b008b834b008d06e900edff3a0085
:101810008482720086827200f707b20087827200ab
:1018200001003200150020001e0490003e0b9000c5
:1018300006035400e63fb0000368a300070032002f
:101840000000a7000500a0008301d1000281d300a1
:101850008180d3000080d3000603e8008301d1001b
:101860000281d3008180d3000080d3000002eb000e
:101870000482d2006400070003f0a1000cf0a7006e
:1018800003f0a0005b003700640247006408e10039
:10189000550032003400be003401be00f6ff3700b0
:1018a0006108e100500032006011b8006000b8002b
:1018b000f1ff370003ff270002002000fbff370085
:1018c000889fbe00830478000300e0002c003500f0
:1018d00003003c0000827000040271002600320008
:1018e00036432000c50020008383cf000a00390062
:1018f0000541b1008283cf00070039000541b100e6
:101900008183cf00040039000541b1008083cf00fe
:10191000010039000541b10085c353006022b800c1
:10192000120032000a003b008482720061026000f3
:101930008301d1000281d3008180d3000080d300d5
:101940000603e8008743e800f7ff3a000700370086
:101950000000400081804800020149008381490065
:101960000603e9008743e900f9ff3a002600070073
:1019700009f0a70003f0a0004f04be00000006001d
:1019800060001000e080180060011900e08119007b
:10199000d3ff3b00033e2c00f7ff370007f0a20007
:1019a000bffe3700680447000294be000094be00ea
:1019b000fc0447008694be008494be0009007800b1
:1019c00066000700080078006400070099007800ae
:1019d000814f70000b003b000800be009300070021
:1019e0004f00b10003003700f3ff2700f2ff2f0084
:1019f0006110b9004f06be004f05be004f04be0087
:101a00000080fa00000006001800200057002000a7
:101a1000080453000d003d000600200097fc2f0035
:101a20000740e1001e003400848272006102600001
:101a30008301d1000281d3008180d3000080d300d4
:101a40000804e800f8ff3a00470020006104600045
:101a500005047400040464000d00320061004000bd
:101a6000e080480060014900e081490003b8a5001a
:101a7000070032000603e8006538e10004003a0080
:101a80008301d1000281d3008180d3000080d30084
:101a9000f87f20000830e1000300350008037800db
:101aa0006000b8006011b8004433dd00f300b200fc
:101ab0008301730000000600889fbe008a9fbe005d
:101ac0008c9fbe000404be000605be00809fbe00c1
:101ad000829fbe0063000700040678000800be0075
:101ae0000a01be005f000700840678004f03be00b5
:101af0004f02be008d4f76007fb097001300330079
:101b0000f0ff2f008b8f6b0006003b000d06660078
:101b10000c00a7000a00370007f0a6001000200004
:101b20000a003700880f5200898f5a008a0f5b0025
:101b30008b8f5b00030039001000200001003e0085
:101b40000000200007f0a7000000ea004f06be00da
:101b50004f05be004f04be00000006008000780064
:101b60005002be005003be004439de00f700b20050
:101b7000f37f200003016100090032000218e10038
:101b800016003a008501720083017300838173009f
:101b90000008200015003a00400020001300370024
:101ba00085017200830173008381730005003a0090
:101bb00004a8be0006a8be00100020000b003700dd
:101bc0000201e9000402420085824a0006034b003c
:101bd00087834b000748a300f9ff32000740a000ad
:101be00004a8be0006a8be002000200080009800c7
:101bf00092009800000006000003be00defb070014
:101c00006220e100020032000600be00050005006f
:101c1000e507b100f107b20004f0230084807000f2
:101c200007f0a70001f0a00024000500e4824000b6
:101c30001078a30007003200640240001178a3006e
:101c40003400be001401be00040032000330a700bf
:101c5000000006003500be001501be000330a000e4
:101c60000000060005ff2700058261000700320022
:101c70000428e100010032002400050006000700ee
:101c800001003a00440005000408050002000700b6
:101c9000f9ff3a00140005006f82610081027000b4
:101ca00085027100850272000000060000017800c4
:101cb00000c2b300010037000201e8009240780042
:101cc00080cf5000fcff3200e9cf5000faff320015
:101cd000d0c2b30080cf500003003a000201e800f8
:101ce00014c0b300050037000042eb00b0c2b300df
:101cf00080cf500001003a000201e8008000eb00b4
:101d000005fd2f00040037006a08b900008041007b
:101d1000850040000201e8009201fb0005804100bf
:101d2000e90f5000f8ff36000404e0000100320023
:101d30008100ea000100780000000600889fbe00d4
:101d40000004be00060037000804e8000000fb00a5
:101d50008900780055000700e10f400004003200c0
:101d6000184078000004e000f7ff3a000000eb00a4
:101d70004f04be0000000600881f7800e1422100e9
:101d8000eeff070000047800e1422100a0002000df
:101d900046000700080078004f04780000000600a5
:101da0008001eb0002003700817178008301e800b8
:101db000828f5100fcff3a0000000600800078008e
:101dc0003004e000feff3a00010050000000e9008e
:101dd00000000600800178000001780031407800a2
:101de000005978000004e000fcff3a00030078008e
:101df00000000600000378008002780002027800ec
:101e00008001eb00080037000402e90063c078009d
:101e1000805a78008301e8000004e00002003a00e4
:101e20008000eb0006003700828f5100f6ff3a0079
:101e3000fbff37000040eb0080f07a008100e800f3
:101e4000848f5000fbff3a00060078000000060077
:101e50000c00fa00889fbe0000047800cfb0970005
:101e6000f0ff2700d0bf9f008004eb0099bf9f00c8
:101e700088bf9f00a8bf9f00200c2000b0bf9f001c
:101e80007881570070805700a60007000fb89700b0
:101e9000094878000fb8970008045000080078003f
:101ea0004f04be000080fa0000000600889fbe00bc
:101eb0000001780001047800b10090000118a3002f
:101ec0003d0032000198a30003003a001800900082
:101ed0000000e00038003a000190a00031049800b2
:101ee00082047800f90fb200180090000000e000b2
:101ef00002003a0028009000000c7800ea8f54009d
:101f000006003a00380090000078a30003003a0071
:101f100088007800d0002000e4ff070098009000bf
:101f200058009000808f50000b0032000100e80044
:101f3000100498001800780009587800000c780008
:101f400011c0b300a044210001487800ea8f54007a
:101f50000600320019003700880078000940780038
:101f60006e050700800478001400370038009000e8
:101f70000088a3001100320018019000a800900012
:101f800048009000a3f9070098009000810f5000ce
:101f900004003200380090000003b30030049800c1
:101fa0008084eb000000eb001004980028009000f3
:101fb000000c7800010037008084eb0009007800f5
:101fc0004f04be0000000600889fbe008a1f7800f4
:101fd000804078000004e00021003d008040ea00dd
:101fe000d0c6b30080cf5000090034008104fb004c
:101ff00042062000110009008204d8000001780088
:10200000010078004311dd006a1f21001f00370026
:102010000100fb00631f210039003700a2002000ef
:10202000110009000200d8000001780001007800ca
:102030004311dd00030141004300dd0003004000c7
:102040003002be002003be0042209000d22090004b
:10205000f22190006221900040fc07002e00370022
:10206000d0c6b30080cf5000230034008104fb00b1
:1020700042062000110009008204d8000001780007
:10208000010078004311dd006a2a21000a014100a5
:10209000a8002000110009000800d8004300dd005e
:1020a0000a00400040229000d0229000602390005f
:1020b000f02390000288900092889000b2899000ee
:1020c0002289900025fc0700801f7800010278001b
:1020d000110009008804d8000102fd004f007800bb
:1020e0000402fb004322dd000a0242005403be004a
:1020f0004402be00d8ff37000100fb00632a210024
:10210000eacf5000c5ff3c004300dd000300400063
:102110005001be004000be004f0578004f04be00d5
:10212000000006008f03b000889fbe008a9fbe009b
:102130008c9fbe008e1f7800e0b79f00f1b79f0014
:1021400082bf9f000000eb00a0b79f00e6043700ad
:102150008001eb0050c2b30080cf50000900320074
:102160000100fb00efb0970050ff0700e10f4000b7
:10217000dd043200afb097008100e800a1b79f00f6
:10218000d90437007fb1970092407800d0c2b300e5
:1021900080cf50000c00320007003c006d40500022
:1021a00080cf50000d0032006b40400080cf5000c7
:1021b00019003a000e00370000c3b30080cf500072
:1021c00015003a000f0037000330a0007fb29700df
:1021d0000402e800f4b79f00eaff37000300a00004
:1021e000ffb297008502e800f5b79f00e5ff3700d2
:1021f0000310a0007fb697000c06e800fcb79f0014
:10220000e0ff37000320a0007fb097000000e80047
:10221000f0b79f00dbff37000318a3000100320076
:102220000300a1000338a300010032000320a10035
:102230000100fb0002fd2f0002004000e90f5000ea
:1022400010003e008000eb00c1b79f000202780042
:102250004fb197006a10b900ffb297001501fb005b
:102260000001410004014100c2b79f005500fb007e
:10227000f5b79f0004004000e90f50000d003e003c
:10228000f3ff37000006eb00ccb79f00a0c2b300fd
:1022900080cf500007003a000fb89700c0007800c8
:1022a00080bf9f00c1b79f007fb197000201e80087
:1022b000f2b79f00e0c2b3007fb29700944f1000c6
:1022c00021003a00830678000de0a0008400e800b9
:1022d00064405000914f100004003200f1b79f009d
:1022e0008002eb00b5b79f00100037000fbe9700cb
:1022f0004c0078008cbf9f00b0b79f00ffb09700e4
:102300008180e800f1b79f00130037003fb29700cb
:102310006a20b9000000410003004000b0b79f00f0
:10232000ffb297008502e800f5b79f007fb69700df
:102330001c01fb0003fd2f0003004100e90f5000ca
:10234000f2ff360004003700830678000dc0a000bd
:102350000000eb00b0b79f007fb19700b24078005b
:10236000f2b79f00c17f9f00c0c6b30080cf50006e
:102370002700320014003c006840500080cf50001d
:102380009d00320009003c006c40500080cf50009e
:10239000290032006b40400080cf500072003200b4
:1023a0000104e000560432008e00370060c6b3001e
:1023b00080cf50001c0032006340400080cf5000ae
:1023c00088003a008c00370030c7b30080cf50003f
:1023d0001c00320007003c006440500080cf5000d9
:1023e000130032000040e80080cf50007d003a002a
:1023f0001100370050c7b30080cf50007d0032007d
:102400006340400080cf500076003a000b00370058
:10241000000028000d48a30001003a000001200040
:1024200080867600ccff37000da0a0007200370038
:102430000d60a000700037000d50a0000d70a000ce
:102440006d0037008fb997004300780083bf9f006d
:10245000000478000000e00001003a00683f21001d
:102460008004eb00010037008104e8008900780057
:10247000088044001004e000fbff3a003fb29700e0
:102480000400e00003003200890f52000100310017
:10249000840478000007eb00cfb29700898f5200c8
:1024a00001003600098752004368de00e106600043
:1024b00019003a000d06780009003700efb09700c8
:1024c0000002200079fe0700e10f40000300320007
:1024d0002fb097000000e800a0b79f000c06e800ae
:1024e0008e0f5600f5ff3a000087eb000a00370018
:1024f000880078003100fb0001047800efb09700fd
:102500006afe0700e10f400003003200afb0970001
:102510008100e800a1b79f000900e900800478006d
:10252000e10f4000f2ff3a000006eb000d00e00072
:102530000a003a00ec033700efb0970000022000d9
:102540005afe0700e10f4000030032002fb1970050
:102550000201e800a2b79f000c06e8008e0f5600ab
:10256000f5ff3a00e00337008fb997004300780089
:1025700083bf9f00cf80de000101780082017800d8
:102580000205be000004be000203be000002be0041
:102590004822de00482edd0004027600c47f9f0042
:1025a0000d48a3000a0032000404e00008003200d5
:1025b000e14f420006003200d1fb2f0001804700ae
:1025c00004487800184098002900200002003700d5
:1025d000d07f9f0019002000d2fb2f00028447000b
:1025e000a6ff3700c3fb2f0003844700190020001b
:1025f000a2ff37000d0cb3000070200000826600bf
:10260000270232000dc8a30002003200640020003f
:10261000b4b79f000d48a300050032000fba970021
:102620004401be004400be0084bf9f000400370088
:102630008fba97004500be0085bf9f003cfb070096
:10264000e0af9f00f1af9f0082b79f0093b79f005c
:102650006022b8006033b8006fa89700ffa8970009
:102660000fb197009fb1970050fb07000000e000fa
:102670000a003d006fa89700ffa897000fb19700d0
:102680009fb1970003f0a200e0af9f00f1af9f0061
:1026900082b79f0093b79f003d00b3000000eb009e
:1026a00080a79f006022b8006033b8006fa8970031
:1026b000ffa897000fb197009fb1970040fb07005c
:1026c0000000e000340032006fa89700ffa89700d8
:1026d0000fb197009fb197003efb070003fc2f004e
:1026e0000381470066fb07000fa097000000e90088
:1026f0006300b900a2002000110009000200d80008
:102700008000fd0081a79f000100e00002003d0065
:102710000100e90080a79f000fa497000840ea008d
:1027200029fe07006faa9700ffaa97000fb3970032
:102730009fb3970089fa0700a0af9f00b1af9f0039
:10274000c2af9f00d3af9f006022b80006002000f8
:1027500007ff230015fb07000000e00002003d001a
:102760000800e9000b0037006022b80006002000d6
:10277000470224002fa89700bfa897004fa99700f1
:10278000dfa9970041fb07000000e00002003500d0
:102790000800e80080a79f003fb29700f80f5200a2
:1027a00057003c00d0c6b300804f520029003600cd
:1027b0000485fb0042062000110009000285d800b4
:1027c00000017800010478004311dd006b1f210037
:1027d0000b0141006022b8000600200007fe230024
:1027e0000288900092889000b2899000228990001f
:1027f0005afa0700a9002000809fbe0011000900be
:102800000984d800000478004f00be004344dd0076
:102810000b04440048229000d822900068239000c6
:10282000f82390004dfa0700801f7800010278001d
:10283000110009000985d8000102fd004f00780051
:102840004322dd000b0242005403be004402be00de
:102850001f0037000480fb00691f2100ea4f52006f
:1028600014003600a2002000110009000280d800e8
:1028700000017800010478004311dd0009014100e6
:102880006022b8000600200007fe230042209000ce
:10289000d2209000f2219000622190002ffa0700d0
:1028a0004344dd00090444003802be002803be0092
:1028b000070037004300dd00090040006022b80037
:1028c0000600200007fe23005001be004000be00ad
:1028d00022fa07000002be000203be006fa89700a4
:1028e000ffa897000fb197009fb19700ecfa07007f
:1028f000e0af9f00f1af9f0082b79f0093b79f00aa
:102900000fa49700e90f540015003c006022b800a6
:102910006033b8006fa89700ffa897000fb1970029
:102920009fb19700a6fa07000000e00032003200d5
:102930006fa89700ffa897000fb197009fb197006d
:1029400054fb0700e00f5000e08f5800e00f5900e3
:10295000e08f590028003a00e10f540026003400af
:102960000400200005002e00b6e02200170124001c
:102970002fa89700bfa897004fa99700dfa997003d
:102980008afa07000000e00002003d0073005400d6
:10299000010037007200540080a79f000fc097000d
:1029a00089fd0700a0af9f00b1af9f00c2af9f009d
:1029b000d3af9f000002be000203be006fa89700c5
:1029c000ffa897000fb197009fb1970062fb070027
:1029d00030fb07000205be000004be006000b80026
:1029e0006011b800a0a79f00b1a79f00c2a79f00d9
:1029f000d3a79f002e0037006fa89700ffa897006d
:102a00000fb197009fb1970022fb07000205be009f
:102a10000004be00e00f5000e08f5800e00f5900a6
:102a2000e08f590002003500a5fb070013003700b6
:102a300010002000010020006011b80008006000b4
:102a4000898060000a0161008b8161008b03d100e5
:102a50000a83d3008982d3000882d3000000720069
:102a600081807200020173008381730094fb070070
:102a70000002be000203be0089fa07000002be0089
:102a80000203be006fa89700ffa897000fb1970040
:102a90009fb19700c1fb0700a0a79f00b1a79f00af
:102aa000c2a79f00d3a79f000000eb0080a79f0054
:102ab00014c0b300653521000b0037000400fb0093
:102ac0004300dd00050040005001be004000be0094
:102ad0000040e10001c8e10002d0e10003d8e100bc
:102ae000030039000442e800f44f5200f3ff3a00bb
:102af000c47f9f000400fb00bfb09700008040002f
:102b00008fa09700010040004fb1970000075100cf
:102b1000bfb197000300e000010032000e07e9009a
:102b200063806600010032000e07e9000d28a30053
:102b300026003200e18066000d18a3000c00320070
:102b4000d00220000100e00001003a000080e9000e
:102b5000efb09700d5fc0700e10f400018003200ed
:102b60002fb297000402e800a4b79f0014003700ba
:102b70000100e00012003200efb0970000022000d8
:102b8000cafc0700e10f40000d003200afb2970011
:102b90008502e800a5b79f0009003700efb0970055
:102ba00000032000c1fc0700e10f400003003200d9
:102bb0002fb697000c06e800acb79f000e07e9009f
:102bc0000e00e000f5ff3c003d0037000d38a3008b
:102bd0000a0032000b003700efb09700000220001f
:102be000b2fc0700e10f4000030032002fb0970055
:102bf0000000e800a0b79f000e07e9000e00e0000b
:102c0000f5ff3c00e18066000d18a3000c003200c7
:102c1000d00220000100e00001003a000080e9003d
:102c2000efb09700a1fc0700e10f40002400320044
:102c3000afb097008100e800a1b79f0020003700e7
:102c40000100e0001e003200efb0970000022000fb
:102c500096fc0700e10f4000190032002fb19700e9
:102c60000201e800a2b79f00150037000000fb003a
:102c70004300dd0061352100010040003002be004c
:102c80002003be000800be000a01be00a2f8070033
:102c9000a4002000050020006033b800a5f807005c
:102ca0000003b000efb0970080fc0700e10f400088
:102cb00003003200afb197008301e800a3b79f0083
:102cc0004f7a97000440e900c07f9f00e14f400029
:102cd000e6ff3a000b003700efb09700000320003a
:102ce00072fc0700e10f400003003200afb2970012
:102cf0008502e800a5b79f000fa097000000e9003b
:102d000080a79f000fa097000000e000f2ff3c00aa
:102d10003fb6970020c1b300f20f560001003c00ff
:102d20006fe09700c07f9f00cf7897000100fb0005
:102d30003fb1970000005100e0a79f000104e000b0
:102d400008003200efb09700e002200057fc0700b7
:102d5000e10f400003003200afb197008301e800ab
:102d6000a3b79f004f78970097fc07000002be00b2
:102d70000203be002fa09700bfa097004fa19700ad
:102d8000dfa19700f5f8070042fa07001e003700a0
:102d90000000fb004300dd006c3521000c0040000a
:102da0003002be002003be000800be000a01be00c3
:102db00059f80700a4002000050020006033b80087
:102dc0005cf807000003b000efb0970037fc070085
:102dd000e10f4000030032002fb297000402e80028
:102de000a4b79f00cf7a97000500fb004300dd00e9
:102df0000c0040003002be002003be000800be00f0
:102e00000a01be004bf807000205be000004be0028
:102e10004f7e97000c40e900c07f9f00e14f4000cb
:102e2000dbff3a000006eb0009003700efb0970027
:102e3000000320001dfc0700e10f400003003200ea
:102e40002fb097000000e800a0b79f000c06e80034
:102e5000efa09700810f5600f4ff3a000d38a30051
:102e6000a10132000e00e0009f0134000006eb00db
:102e7000efb09700000220000cfc0700e10f4000bb
:102e8000030032002fb197000201e800a2b79f00b3
:102e90000c06e8008e0f560093013200f4ff370055
:102ea0000d007800000cb20028003a000d00e00090
:102eb00005003d008fb997004305be004304be00e6
:102ec00083bf9f00140037000d48a3000b003200a1
:102ed0000fba97004400be0084bf9f004f89de00f8
:102ee000cf91de000002be0002037800820378006a
:102ef0000605be000404be00070037008fba970025
:102f00004500780085bf9f0000047800cfc4de0034
:102f1000090578008a057800e00f5400e08f5c0016
:102f2000e00f5d00e08f5d0020003d003d00b3003c
:102f30006000b8006011b80008045000898458008f
:102f40000a0559008b855900180037000d00e00074
:102f500005003d000fbe97004c05be004c04be00ae
:102f60008cbf9f00110037000d48a30008003200fd
:102f70008fba97004500be0085bf9f00040178000e
:102f8000840178000205be000004be00070037007f
:102f90000fbe97004c0078008cbf9f0000047800a3
:102fa000090020000a0020000b0020003fb097001d
:102fb0000000e00007003a00e00f5400e08f5c00e2
:102fc000e00f5d00e08f5d0002003a00110020007c
:102fd000b1b79f000d0778000e0cb200000420006e
:102fe000800f57002f00320003003c000e00e0006d
:102ff000070032003f00370000082000800f570014
:1030000014003200000c2000800f570039003a00f5
:1030100014c0b300653521000b0037000400fb002d
:103020004300dd00050040005001be004000be002e
:103030000040e10001c8e10002d0e10003d8e10056
:103040002b0039000442e800f44f5200f3ff3a002d
:103050002700370000012000010020006011b800a7
:1030600014c0b3000040e10001c8e10002d0e1005b
:1030700003d8e1001e003900450020000000d00008
:103080008180d2000281d2008381d2008502e900d2
:10309000faff3a000442e800f04f5200f1ff3a0014
:1030a0001300370080002000010020006011b800ec
:1030b00014c0b3000040e10001c8e10002d0e1000b
:1030c00003d8e1000a0039003c0020000000d000d5
:1030d0008180d2000281d2008381d2000c06e900f7
:1030e000faff3a000442e800f54f5200f1ff3a00bf
:1030f000c47f9f00cf7897000100fb003fb197008d
:10310000820f500002003d00c27f9f000400370084
:10311000bfb19700808f510001003d00b0b79f0004
:103120004fb297000400e0000400320063806600a4
:10313000020032000402e900c4b79f000de8a300ba
:103140000b003200cfb297003fb697008c8f520031
:1031500003003c000000eb00c0b79f0004003700f4
:10316000cfb097003fb1970082805000c1b79f0059
:10317000cf7997000300fb000002eb0094a79f00ab
:10318000cfb29700808f52000200340000805200be
:1031900090a79f000d28a30037003200e180660051
:1031a0000d18a3000c003200d00220000100e00046
:1031b00001003a000080e900efb097003bfb0700f8
:1031c000e10f40000e0032002fb697000c06e80019
:1031d000acb79f000a0037000100e0000800320091
:1031e000efb097000002200030fb0700e10f400025
:1031f000030032002fb097000000e800a0b79f0046
:103200009fa097000100e0000f0032000006eb00d5
:10321000efb097000003200024fb0700e10f4000ff
:10322000030032002fb197000201e800a2b79f000f
:103230000c06e8009fa19700830f5600f4ff3a00a8
:103240000002eb0094a79f00bfb29700c328dd00e7
:10325000e03421008080400091af9f004228dd00d3
:103260006400500080af9f006328b900f0a79f0062
:1032700063065000820037001fa697000c00e00094
:1032800011003200688066000f003a0000067800e6
:10329000efb097000002200004fb0700e10f4000a0
:1032a000030032002fb097000000e800a0b79f0095
:1032b0000c06e8009fa09700810f5600f4ff3a002b
:1032c0000001eb0092a79f00e18066000d18a300ab
:1032d0000c003200d00220000100e00001003a00a2
:1032e0000080e900efb09700f0fa0700e10f40001e
:1032f000d5ff3200afb197008301e800a3b79f006c
:10330000d1ff37000100e000cfff3200efb097009f
:1033100000022000e5fa0700e10f4000caff32007a
:103320002fb297000402e800a4b79f00c6ff370041
:1033300000042000800f57003000320003003c00e2
:103340000e00e000070032003d00370000082000ba
:10335000800f570011003200000c2000800f570032
:1033600037003a001fa897003002be002003be00bd
:103370000800be000a01be00e7f60700a400200016
:10338000050020006033b800eaf6070004c3b3006c
:1033900004424000c47f9f0029003700d53f210030
:1033a000d5b79f000d58a30002003a00e04021006d
:1033b000d0b79f0014002000050020006033b80043
:1033c0008fa897008100e900050033000402d000b7
:1033d0008582d2000683d2008783d200f9ff3700ae
:1033e0000800be000a01be00cbf607006f006000b7
:1033f0005fb1970062407800100037001400200091
:10340000050020006033b8008c0178008301e900da
:10341000050033000402d0008582d2000683d2006a
:103420008783d200f9ff37000800be000a01be0002
:10343000b9f60700674060000043b000c07f9f00fe
:103440004f7a97000400fb00efb0970097fa07004f
:10345000e10f400003003200afb297008502e800a0
:10346000a5b79f001fa897006800500090af9f006d
:103470008fa89700e480500081af9f00630656003c
:10348000d0ff2f003fb197000090b900ffa1970037
:103490000080410063005000800f5600a4ff3a00f6
:1034a0000d38a300100032001fa297000400e000b6
:1034b0000d0034000006eb00efb097000002200082
:1034c0007afa0700e10f400003003200afb2970024
:1034d0008502e800a5b79f000c06e8001fa0970032
:1034e000800f5600f4ff3a007fb19700b240780099
:1034f000f2b79f00c17f9f000104e00014fb3a0077
:103500002fb097004f0778004f06be004f05be0052
:103510004f04be008f03b100000006000200fa0055
:10352000889fbe00a0ff9f0001047800b1009000ba
:10353000810478000904b200020032000000fb00a0
:10354000360037000118a30005003a000103b3005c
:1035500031049800190498000080eb002f00370018
:10356000580090000000e00006003a00480090007b
:1035700012002000e680570026f407001904980086
:1035800024003700280090000000e00008003a0006
:103590006044210020049800000c780020002000e6
:1035a00050049800100498000130a00031049800e5
:1035b00018019000a80090004800900015f4070042
:1035c00028009000000c78000080eb0010049800a8
:1035d00018007800aff8970001587800000c7800c8
:1035e0002ff89700ea4f50000a003a003800900088
:1035f0000088a3000700320018019000a800900086
:103600004800900003f4070019049800a8009000f7
:10361000010c7800aff897000100fb004f04be00da
:083620000080fa000000060022
:020000040000fa
:020000040001f9
:0457f0003fff000077
:020000040000fa
:020000040001f9
:0457f400c21c0000d3
:020000040000fa
:020000040001f9
:0457f800bdfa0000f6
:020000040000fa
:020000040001f9
:0457fc007f3f0000eb
:020000040000fa
:10000800dc020000dc020000dc020000dc02000070
:10001800dc020000dc020000dc020000dc02000060
:10002800dc020000dc020000dc020000dc02000050
:10003800dc020000dc020000dc0200009a42000042
:10004800dc020000dc0200005e370000183b000004
:10005800003b0000dc020000dc020000dc020000c3
:10006800dc020000dc020000dc020000dc02000010
:10007800dc020000dc020000dc020000dc02000000
:10008800dc020000dc020000dc020000dc020000f0
:10009800dc020000dc020000dc020000dc020000e0
:1000a800dc020000dc020000dc020000dc020000d0
:1000b800dc020000dc020000dc020000dc020000c0
:1000c800dc020000dc020000dc020000dc020000b0
:1000d800dc020000dc020000dc020000dc020000a0
:1000e800dc020000dc020000dc020000dc02000090
:1000f800dc020000dc020000dc020000dc02000080
:10010800dc020000dc020000dc020000dc0200006f
:10011800dc020000dc020000dc020000dc0200005f
:10012800dc020000dc020000dc020000dc0200004f
:10013800dc020000dc020000dc020000dc0200003f
:10014800dc020000dc020000dc020000dc0200002f
:10015800dc020000dc020000dc020000dc0200001f
:10016800dc020000dc020000dc020000dc0200000f
:10017800dc020000dc020000dc020000dc020000ff
:10018800dc020000dc020000dc020000dc020000ef
:10019800dc020000dc020000dc020000dc020000df
:1001a800dc020000dc020000dc020000dc020000cf
:1001b800dc020000dc020000dc020000dc020000bf
:1001c800dc020000dc020000dc020000dc020000af
:1001d800dc020000dc020000dc020000dc0200009f
:1001e800dc020000dc020000dc020000dc0200008f
:0801f800dc020000dc02000043
:020000040000fa
:10020800dc020000dc020000dc020000dc0200006e
:10021800dc020000dc020000dc020000dc0200005e
:10022800dc020000dc020000dc020000dc0200004e
:10023800dc020000dc020000dc0200009a42000040
:10024800dc020000dc0200005e370000183b000002
:10025800003b0000dc020000dc020000dc020000c1
:10026800dc020000dc020000dc020000dc0200000e
:10027800dc020000dc020000dc020000dc020000fe
:10028800dc020000dc020000dc020000dc020000ee
:10029800dc020000dc020000dc020000dc020000de
:1002a800dc020000dc020000dc020000dc020000ce
:1002b800dc020000dc020000dc020000dc020000be
:1002c800dc020000dc020000dc020000dc020000ae
:1002d800dc020000dc020000dc020000dc0200009e
:1002e800dc020000dc020000dc020000dc0200008e
:1002f800dc020000dc020000dc020000dc0200007e
:10030800dc020000dc020000dc020000dc0200006d
:10031800dc020000dc020000dc020000dc0200005d
:10032800dc020000dc020000dc020000dc0200004d
:10033800dc020000dc020000dc020000dc0200003d
:10034800dc020000dc020000dc020000dc0200002d
:10035800dc020000dc020000dc020000dc0200001d
:10036800dc020000dc020000dc020000dc0200000d
:10037800dc020000dc020000dc020000dc020000fd
:10038800dc020000dc020000dc020000dc020000ed
:10039800dc020000dc020000dc020000dc020000dd
:1003a800dc020000dc020000dc020000dc020000cd
:1003b800dc020000dc020000dc020000dc020000bd
:1003c800dc020000dc020000dc020000dc020000ad
:1003d800dc020000dc020000dc020000dc0200009d
:1003e800dc020000dc020000dc020000dc0200008d
:0803f800dc020000dc02000041
:020000040000fa
:103628004d4500004f5700000d0a000000690000da
:103638006e310000203d000020250000642c0000b1
:10364800206900006e320000203d000020250000a7
:10365800642c0000206900006e330000203d00004b
:1036680020250000640d00000a0000004249000007
:103678005420000025640000204900005320000069
:10368800484900000d0a00000042000049540000ab
:10369800202500006420000049530000204c000051
:1036a8004f0d00000a0000005350000049200000a0
:1036b8004952000051200000434f0000554e0000c1
:1036c800542000003d200000257500000d0a000070
:1036d8000053000050490000204300004d44000002
:1036e800204300004f5500004e540000203d0000cc
:1036f80020250000750d00000a000000535000004e
:1037080049200000494e0000464f000020430000b9
:103718004f5500004e540000203d000020250000b9
:10372800750d00000a0000005350000049200000f9
:103738005245000041440000204300004f5500005e
:103748004e540000203d000020250000750d0000ab
:103758000a000000535000004920000057520000a2
:103768004954000045200000434f0000554e00001a
:10377800542000003d200000257500000d0a0000bf
:103788000053000050490000204f0000564500003b
:10379800524600004c4f00005720000042490000ec
:1037a80054200000203d0000203100000d0a0000d8
:1037b8000053000050490000204f0000564500000b
:1037c800524600004c4f00005720000042490000bc
:1037d80054200000203d0000203000000d0a0000a9
:1037e80000530000504900003153000054410000cc
:1037f800542000003d2000003078000025300000f3
:10380800345800000d0a0000005f0000535000000b
:103818004931000049460000203d000020310000e9
:103828000d0a0000005f00005350000049310000fd
:1038380049460000203d0000203000000d0a00002d
:10384800005f000053500000493100004945000066
:10385800203d0000203100000d0a0000005f00003c
:10386800535000004931000049450000203d000048
:10387800203000000d0a0000000d00000a52000070
:1038880065740000757200006e6500006420000019
:10389800566100006c750000652000003d200000a6
:1038a800256600000d0a0000006100006e6100003e
:1038b8006c6f000067310000203d000020250000eb
:1038c800640d00000a000000616e0000616c0000d9
:1038d8006f670000322000003d20000025640000d2
:1038e8000d0a0000006100006e6100006c6f0000ae
:1038f80067330000203d000020250000640d000013
:103908000a000000616e0000616c00006f67000033
:10391800342000003d200000256400000d0a00004e
:10392800006100006e6100006c6f000067350000e8
:10393800203d000020250000640d00000a00000062
:10394800616e0000616c00006f67000036200000a7
:103958003d200000256400000d0a0000005400000e
:10396800656d000070200000536500006e73000054
:103978006f720000205b00004a3600005d200000e6
:1039880069730000202500006420000064650000c1
:103998006772000065650000730d00000a000000f2
:1039a800546500006d70000020530000656e000033
:1039b800736f0000722000005b4a0000375d000052
:1039c80020690000732000002564000020640000c6
:1039d8006567000072650000657300000d0a00004d
:1039e80000540000656d0000702000005365000061
:1039f8006e7300006f720000205b00004a38000000
:103a08005d2000006973000020250000642000008c
:103a1800646500006772000065650000730d0000b2
:103a28000a000000546500006d700000205300007b
:103a3800656e0000736f0000722000005b4a000092
:103a4800395d000020690000732000002564000033
:103a5800206400006567000072650000657300005f
:103a68000d0a000000540000656d00007020000081
:103a7800536500006e7300006f720000205b000049
:103a88004a310000335d0000206900007320000007
:103a9800256400002064000065670000726500006e
:103aa800657300000d0a000000540000656d0000f9
:103ab80070200000536500006e7300006f720000f4
:103ac800205b00004a310000355d000020690000dd
:103ad8007320000025640000206400006567000072
:103ae80072650000657300000d0a000000540000b4
:103af800656d000070200000536500006e730000c3
:103b08006f720000205b00004a310000365d000043
:103b18002069000073200000256400002064000074
:103b28006567000072650000657300000d0a0000fb
:103b380000540000656d000070200000536500000f
:103b48006e7300006f720000205b00004a310000b5
:103b5800375d000020690000732000002564000024
:103b6800206400006567000072650000657300004e
:103b78000d0a0000002500007525000075250000cd
:103b880075250000750d00000a0000006163000043
:103b980074530000657400005374000075620000df
:103ba800436d000064280000292000003d2000002b
:103bb800256400000d0a000000000000000000005d
:103bc80000000000000000000000000000000000ed
:103bd80000000000000000000000000000000000dd
:103be80000000000000000000000000000000000cd
:103bf80000000000000000000000000000000000bd
:103e3800000000000000000000000000202000003a
:103e4800202000002000000047450000540000002a
:103e58005345000054000000434c00004541000059
:103e6800527c0000434c0000520000005245000004
:103e78005345000054000000484500004c4c000029
:103e88004f2000004b490000545400005900000026
:103e980053500000493200005445000053540000bc
:103ea80000000000289f0000982100002c9f0000bf
:103eb800a8210000309f0000b82100003a9f0000b0
:103ec800c8210000409f0000d42100004c9f000042
:103ed800e6210000559f000000000000434100005b
:103ee80052440000204900004e4600004f000000e8
:103ef8005350000049200000535400004154000072
:103f080053000000444900004e000000444f0000e8
:103f180055540000004100004443000000540000d4
:103f2800454d00005000000041440000434200009d
:103f38005553000059000000434f00004d50000049
:103f48004153000053000000729f00003622000019
:103f58007c9f0000bc220000869f000044220000d5
:103f68008a9f0000802200008f9f0000fe2400002e
:103f7800939f0000bc260000989f00001c280000aa
:103f8800a09f000094230000559f0000000000003f
:103f98005354000055420000004300005300000045
:103fa800cc9f00005e2800008a9f00008228000045
:103fb800d19f000098280000559f000000000000d5
:103fc8007c9f0000ac2800008a9f0000c2280000e7
:103fd800559f000000000000485500004d300000cb
:103fe80031000000485500004d300000320000004c
:103ff800485500004d3000003300000048550000cf
:104008004d3000003400000046490000424f0000d7
:1040180000540000454d0000503000003100000001
:10402800544500004d50000030320000005400009c
:10403800454d00005030000033000000544500009a
:104048004d5000003034000000540000454d000081
:104058005030000035000000544500004d5000006d
:104068003036000000540000454d0000503000007c
:1040780037000000544500004d5000003038000063
:1040880000480000323000005f31000000480000a6
:10409800323000005f32000000480000323000007b
:1040a8005f33000000480000323000005f34000039
:1040b80000000000f09f0000f69f0000fc9f000039
:1040c80002a0000008a000000da0000014a000003d
:1040d8001ba0000022a0000029a0000030a00000c2
:1040e80037a000003ea0000045a000004ba0000043
:1040f80051a0000057a0000000000000454e00003d
:1041080056520000004900004e540000455300007c
:1041180054000000313500003a320000383a0000ff
:1041280030300000004a0000756c000020200000bc
:10413800322000003230000031320000000d000053
:104148000a4600004f430000452000004348000095
:10415800415300005349000053200000454e000021
:1041680056490000524f00004e4d0000454e0000d9
:10417800544100004c200000424f00004152000012
:104188004420000042750000696c000074200000a3
:104198006f6e00002025000073200000617400008d
:1041a80020250000730d00000a00000020200000f8
:1041b800202000002000000045520000522000008e
:1041c80025300000346400000d0a00000052000091
:1041d800445900000d0a000000000000436100007f
:1041e800726400002054000079700000653a0000f5
:1041f80020250000640d00000a0000004361000053
:1042080072640000204e0000616d0000653a0000f5
:1042180020250000730d00000a0000005661000010
:1042280072690000616200006c650000204e0000a9
:10423800616d0000657300003a0d00000a0000007f
:10424800286900006e70000075740000290d0000d8
:104258000a000000286f00007574000070750000e7
:10426800742900000d0a000000280000696e000093
:104278006f750000742900000d0a0000000d000091
:104288000a0000000000000000000000000000001c
:104298000000000000000000000000000000000016
:1042a8000000000000000000000000000000000006
:1042b80000000000000000000000000000000000f6
:1042c80000000000000000000000000000000000e6
:1042d80000000000000000000000000000000000d6
:1042e800000000004255000046200000425900002e
:1042f80054450000204900005320000046550000a6
:104308004c4c00000d0000002009000000200000b7
:104318000030000031320000333400003536000030
:084328003738000039000000e5
:020000040000fa
:104330000200fa00000f78005200200081fa2900e4
:104340001e007800740f07000080fa0000000600cd
:104350000200fa00000f78005200200041fd290001
:104360001e0078006c0f07000080fa0000000600b5
:104370000200fa00000f78005200200041fe2900e0
:104380001e007800640f07000080fa00000006009d
:104390000200fa00000f78000000fe000000eb00b1
:1043a0000080fa00000006000200fa00000f78000a
:1043b000c0d6200041b1290006000900315878001c
:1043c0000000eb000080fa00000006000800fa0080
:1043d000300798000040eb00404798000040eb0099
:1043e000304798000040eb002047980080002000f4
:1043f0006f03070070c8b300e81207000000000058
:104400000040eb00e5120700404798000040eb0039
:10441000e2120700304798000040eb00df1207006f
:10442000204798002e4090008080fb003e40900086
:104430000081fb004e4090000080fb00811f78004f
:10444000821f7800801f7800b0b12900801f78009b
:1044500000ab20007ef60700e887570001ab200084
:1044600010002000da0b0700e0ff37000200fa001e
:10447000000f7800e0e620004e1107000000eb007e
:104480000080fa00000006000400fa0010079800ff
:104490001e00900005f60700000f78001e0078004f
:1044a000210707000000e000080032001e0078002d
:1044b000801f7800a0b32900801f7800c0d620009c
:1044c00063f60700e4875700070037001e007800f6
:1044d000801f780090b42900801f7800c0d620008b
:1044e0005bf60700e4875700c1d6200010002000cb
:1044f000b70b07000000eb000080fa000000060088
:104500000400fa00100798001e009000e7f507006d
:10451000000f78001e0078004d0607000000e00044
:10452000080032001e007800801f7800a0b3290028
:10453000801f7800c0d6200045f60700e4875700aa
:10454000070037001e007800801f780090b4290013
:10455000801f7800c0d620003df60700e487570092
:10456000c1d6200010002000990b07000000eb00ce
:104570000080fa00000006000400fa00100798000e
:10458000e6090700000f78001e007800801f780001
:1045900080b52900801f780000ab20002cf60700b2
:1045a000e487570001ab200010002000880b0700b3
:1045b000de090700000f78001e007800801f7800d9
:1045c000d0b62900801f780000ab200020f607003d
:1045d000e487570001ab2000100020007c0b07008f
:1045e000d6090700000f78001e007800801f7800b1
:1045f00020b82900801f780000ab200014f60700c7
:10460000e487570001ab200010002000700b07006a
:10461000ce090700000f78001e007800801f780088
:1046200080b92900801f780000ab200008f6070041
:10463000e487570001ab200010002000640b070046
:10464000c6090700000f78001e007800801f780060
:10465000e0ba2900801f780000ab2000fcf50700bd
:10466000e487570001ab200010002000580b070022
:1046700040c2bf000044b2000004e0000400320069
:1046800051bc290010002000510b07000300370027
:10469000d1bd2900100020004d0b07000012800042
:1046a000801f780050bf2900801f780000ab2000d9
:1046b000e7f50700e487570001ab20001000200059
:1046c000430b070085c0bf00644060000004e000a9
:1046d0000400320091c02900100020003c0b0700ac
:1046e0000300370071c1290010002000380b0700bb
:1046f00095c0bf00644060000004e0000400320088
:1047000051c2290010002000310b070003003700c0
:1047100031c32900100020002d0b07000000eb0022
:104720000080fa00000006001800fa00200f980030
:104730002e0890005df50700100f98000000eb00b8
:10474000000f98006000b80060079800710798009b
:104750000000eb00500798000000eb0040079800b5
:104760000000eb00300798000000eb0020079800e5
:104770000000eb00100798000000eb00000f78002d
:104780001e089000300f9800be089000e18f500086
:10479000110032003e089000e10f500004003c0080
:1047a000be0890000100e00008003200120037004f
:1047b0003e089000e20f50000a003200be08900050
:1047c000e38f50000a0032000b0037006009200020
:1047d000000f980008003700600d2000000f9800bf
:1047e00005003700600a2000000f98000200370023
:1047f000600e2000000f980060c2a80000000000ba
:10480000900020006a0207000e089000e3110700e4
:10481000000000000040eb00e01107005007980086
:104820000040eb00dd110700400798000040eb005e
:10483000da11070030079800300620005c020700fc
:104840005e009000200798002e0090004800dd00d8
:1048500020079800ce009000f00f200080806000bc
:104860002e00900001007000200798002e0090009c
:1048700000004000200798003e0090004700de0046
:10488000300798000000eb00100798001e00900011
:104890004800dd0010079800be009000f00f2000d7
:1048a000808060001e0090000100700010079800da
:1048b000ae0090001e009000008f700022002000cb
:1048c0009e0078001e089000760c07006007980094
:1048d000710798006e009000fe009000809fbe005f
:1048e00010c42900801f7800c0d6200058f50700aa
:1048f000e6875700c1d6200010002000b40a070048
:10490000de009000811f780090c52900801f78008c
:10491000c0d620004ef50700e4875700c1d620001e
:1049200010002000aa0a07004e009000801f7800a7
:1049300080c62900801f7800c0d6200044f50700fb
:10494000e4875700c1d6200010002000a00a07000d
:10495000be009000811f780070c72900801f78007a
:10496000c0d620003af50700e4875700c1d62000e2
:1049700010002000960a07002e009000801f78008b
:1049800060c82900801f7800c0d6200030f50700dd
:10499000e4875700c1d62000100020008c0a0700d1
:1049a0009e009000811f780050c92900801f780068
:1049b000c0d6200026f50700e4875700c1d62000a6
:1049c00010002000820a07001e007800801f780077
:1049d00040ca2900801f7800c0d620001cf50700bf
:1049e000e4875700c1d6200010002000780a070095
:1049f0000000eb000080fa00000006001c00fa0036
:104a0000300f98003e089000a8f40700200f98008f
:104a10000000eb00100f98000000eb00000f980062
:104a20000000eb00700798000000eb0060079800a2
:104a30000000eb00500798000000eb0040079800d2
:104a40000000eb00300798006000b80010079800e5
:104a5000210798000000eb00000f78002e0890005e
:104a6000e80f500003003c0080002000000f780099
:104a70000200370090002000000f78002e08900000
:104a80006101b900420f9800530f9800b000200058
:104a9000010020004e099000de099000800f5100b7
:104aa000818f590032003e004e089000de089000d1
:104ab000006001000b0037000d0037000f003700c9
:104ac00011003700130037001500370017003700ba
:104ad000190037001b0037001d0037001f0037008a
:104ae00021003700600820003007980020003700c0
:104af000600c2000300798001d003700600920007e
:104b0000300798001a003700600d20003007980029
:104b100017003700600a20003007980014003700a3
:104b2000600e20003007980011003700600b200055
:104b3000300798000e003700600f20003007980003
:104b40000b0037006009200030079800080037008c
:104b5000600a20003007980005003700600520003b
:104b60003007980002003700600d200030079800e1
:104b70001e0078008e01070060c2a800000000003f
:104b80003e00900005110700000000000040eb000f
:104b900002110700100f98000040eb00ff10070003
:104ba000000f98000040eb00fc1007007007980011
:104bb000300620007e0107009e08900061079800e3
:104bc0006e0090004800dd00600798008e0890009d
:104bd000f00f2000808060006e00900001007000e7
:104be000600798006e009000000040006007980089
:104bf0007e0090004700de00700798000000eb0088
:104c0000500798005e0090004800dd0050079800b3
:104c1000fe009000f00f2000808060005e00900099
:104c20000100700050079800ee0090005e009000b8
:104c3000008070004007980022002000ce00900005
:104c40002e089000970b0700100798002107980086
:104c50001e019000ae019000829fbe0010c429008a
:104c6000801f7800c0d6200079f40700e68757003f
:104c7000c1d6200010002000d50907009e09900031
:104c8000831f780090c52900801f7800c0d62000bf
:104c90006ff40700e4875700c1d620001000200001
:104ca000cb0907000e089000801f780080c62900fd
:104cb000801f7800c0d6200065f40700e487570005
:104cc000c1d6200010002000c1090700fe0090009e
:104cd000811f780070c72900801f7800c0d620008f
:104ce0005bf40700e4875700c1d6200010002000c5
:104cf000b70907006e019000821f780060c8290084
:104d0000801f7800c0d6200051f40700e4875700c8
:104d1000c1d6200010002000ad090700de01900080
:104d2000831f780050c92900801f7800c0d620005a
:104d300047f40700e4875700c1d620001000200088
:104d4000a30907004e009000801f780040ca290088
:104d5000801f7800c0d620003df40700e48757008c
:104d6000c1d6200010002000990907000000eb00c8
:104d70000080fa00000006000800fa0020079800f2
:104d80002e009000c9f30700100798000000eb0008
:104d9000000f78001e009000300798003e00900041
:104da000e30f50004d0032003e009000e30f500032
:104db0000a003c003e009000e10f50002500320048
:104dc0003e009000e10f500033003c003e00900098
:104dd0000000e0000e003200940037003e0090001a
:104de000e50f50005f0032003e009000e50f5000dc
:104df0004b0035003e009000e60f50006a00320084
:104e00003e009000e70f5000780032008700370026
:104e100002002c00934724000000eb00eb02070087
:104e200033ee0700000f78001e007800801f780026
:104e300030cb2900801f7800c0d6200004f4070082
:104e4000e4875700c1d62000100020006009070049
:104e50007600370002002c00934724001000200049
:104e6000da02070022ee0700000f78001e0078002b
:104e7000801f780040cd2900801f7800c0d6200018
:104e8000f3f30700e4875700c1d62000100020008c
:104e90004f0907006500370002002c0093472400eb
:104ea00020002000c902070011ee0700000f780063
:104eb0001e007800801f780050cf2900801f7800e6
:104ec000c0d62000e2f30700e4875700c1d62000d7
:104ed000100020003e0907005400370002002c009b
:104ee0009347240030002000b802070000ee0700be
:104ef000000f78001e007800801f780060d1290024
:104f0000801f7800c0d62000d1f30700e487570047
:104f1000c1d62000100020002d09070043003700f3
:104f200002002c009347240040002000a702070045
:104f3000efed0700000f78001e007800801f78005a
:104f400070d32900801f7800c0d62000c0f307006e
:104f5000e4875700c1d62000100020001c0907007c
:104f60003200370002002c0093472400500020003c
:104f700096020700deed0700000f78001e007800a3
:104f8000801f780090d52900801f7800c0d62000af
:104f9000aff30700e4875700c1d6200010002000bf
:104fa0000b0907002100370002002c009347240062
:104fb0006000200085020700cded0700000f78009b
:104fc0001e007800801f7800b0d72900801f78006d
:104fd000c0d620009ef30700e4875700c1d620000a
:104fe00010002000fa0807001000370002002c0013
:104ff000934724007000200074020700bced0700f6
:10500000000f78001e007800801f7800d0d929009a
:10501000801f7800c0d620008df30700e48757007a
:10502000c1d6200010002000e90807000000eb00b6
:105030000080fa00000006000a00fa00400798000d
:105040000000eb0038040700000f7800100020007b
:1050500035040700100798002000200032040700e4
:1050600020079800300020002f0407003007980028
:105070003e009000ae0090001e0190009e0178005e
:10508000801f7800811f7800821f7800831f7800be
:10509000f0db2900801f780000ab20006cf30700d4
:1050a000ea87570001ab200010002000c808070065
:1050b0000000eb000080fa00000006000400fa0087
:1050c000100798001e009000f8f20700000f78000b
:1050d0001e007800801f7800a0dc2900801f780067
:1050e000c0d620005af30700e487570001ab200028
:1050f00010002000b60807000000eb000080fa0056
:10510000000006000400fa00100798001e0090003e
:10511000e6f20700000f7800110020001e00780062
:10512000960207000000eb000080fa000000060075
:105130000400fa00100798001e009000dbf2070040
:10514000000f78001e007800190007000000eb0037
:105150000080fa00000006000200fa00000f78004c
:10516000060707000a0707000e07070012070700d7
:105170001607070040c2a9000000eb000080fa00fb
:10518000000006000400fa00100798001e009000be
:10519000c6f20700000f78008000eb001e007800c8
:1051a000760207000000eb000080fa000000060015
:1051b0000600fa00000f78001e0078006101b900b7
:1051c00012079800230798003006200001002000f5
:1051d0001e019000ae019000800f5100818f590098
:1051e000f6003e001e009000ae009000006001003e
:1051f000630037006f0037007b00370087003700ff
:10520000930037009f003700ab003700b70037002e
:10521000c3003700cf003700e8003700e700370051
:10522000e6003700e5003700e4003700e300370010
:10523000e2003700e1003700e0003700df00370010
:10524000de003700dd003700dc003700db00370010
:10525000da003700d9003700d8003700d700370010
:10526000d6003700d5003700d4003700d300370010
:10527000d2003700d1003700d0003700cf00370010
:10528000ce003700cd003700cc003700cb00370010
:10529000ca003700c9003700c8003700c700370010
:1052a000c6003700c5003700c4003700c300370010
:1052b000c2003700c1003700c0003700bf00370010
:1052c000be003700bd003700bc003700bb00370010
:1052d000ba003700b9003700b8003700b700370010
:1052e000b6003700b5003700b4003700b300370010
:1052f000b2003700b1003700b0003700af00370010
:10530000ae003700ad003700ac003700ab0037000f
:10531000aa003700a9003700a8003700a70037000f
:10532000a6003700a5003700a4003700a30037000f
:10533000a2003700a1003700a00037009f0037000f
:105340009e0037009d0037009c0037009b0037000f
:105350009a0037009900370098003700970037000f
:10536000960037009500370094003700930037000f
:10537000920037009100370090003700820037001c
:105380008000eb000000eb00fc0107008000eb0058
:1053900010002000f90107008000eb002000200031
:1053a000f60107008000eb0030002000f301070049
:1053b0008e003700110020000000eb00ef01070015
:1053c0008000eb0010002000ec0107008000eb00e3
:1053d00020002000e90107008000eb0030002000e1
:1053e000e6010700810037008000eb000000eb00c1
:1053f000e20107001100200010002000df0107007b
:105400008000eb0020002000dc0107008000eb00a2
:1054100030002000d901070074003700110020007f
:105420000000eb00d5010700110020001000200053
:10543000d20107008000eb0020002000cf01070010
:105440008000eb0030002000cc010700670037002f
:105450008000eb000000eb00c80107008000eb00bb
:1054600010002000c50107001100200020002000ce
:10547000c20107008000eb0030002000bf010700e0
:105480005a003700110020000000eb00bb010700ac
:105490008000eb0010002000b80107001100200080
:1054a00020002000b50107008000eb003000200044
:1054b000b20107004d0037008000eb000000eb0058
:1054c000ae0107001100200010002000ab01070012
:1054d0001100200020002000a80107008000eb0040
:1054e00030002000a5010700400037001100200017
:1054f0000000eb00a10107001100200010002000b7
:105500009e01070011002000200020009b010700e1
:105510008000eb00300020009801070033003700c6
:105520008000eb000000eb00940107008000eb001e
:1055300010002000910107008000eb0020002000f7
:105540008e01070011002000300020008b010700b1
:1055500026003700110020000000eb008701070043
:105560008000eb0010002000840107008000eb00a9
:1055700020002000810107001100200030002000e1
:105580007e01070019003700110020000000eb0029
:105590007a010700110020001000200077010700a9
:1055a00011002000200020007401070011002000dd
:1055b00030002000710107000c00370011002000ae
:1055c0000000eb006d01070011002000100020001a
:1055d0006a01070011002000200020006701070079
:1055e0001100200030002000640107000080fa0054
:1055f000000006001000fa00500798000000eb00c1
:10560000400798000000eb00300798000000eb0016
:10561000200798006000b800008fbe005e00900078
:10562000e70f50000200340070002000500798007f
:1056300060c2a9005e009000ddfe07000040eb00a4
:10564000560e0700400798000040eb00530e07007d
:105650003007980000000000a0002000d4fe0700e2
:105660004e009000200798002e0090004500dd00bd
:1056700020079800be009000800f2000008060008e
:10568000300798003e0090004300de00300798008d
:10569000be009000f00f2000808060002e0090007f
:1056a00001007000200798002e009000cf80de00df
:1056b00030ec070060079800710798002e009000fa
:1056c0000000e00007003d000200200003782400f5
:1056d0006e009000fe00900052ec070060079800fa
:1056e000710798000200200003e823006e0090007c
:1056f000fe009000a8ec0700008fbe001e01be0057
:105700005e009000030007001e00be000080fa004b
:10571000000006004e00fa00889fbe008a1f780035
:105720004027980052279800632798006800470098
:1057300021e029000f000900311878000002b100b3
:105740006000b80020079800310798008002200010
:105750000e00400022de29000f00090032187800f8
:105760000002b1000000eb00100798000000eb0001
:10577000000f78004e209000800040000080200044
:105780000080400010007800f30f50002c0034001f
:105790000000eb00000f7800110037004e2290004f
:1057a0009e0278004e2090001e01e8007400b900af
:1057b00002004000c200dd000081200000804000a7
:1057c0001001be007420b90005004000c200dd00d9
:1057d00000812000008040000288be001e0fe8000b
:1057e000330120009e8f1100ecff34004e2090000a
:1057f00080004000008020008080400030012000b8
:1058000080087800ce2190004e209000800040005b
:105810000080200000804000100178007418b9005a
:1058200002004000c200dd00008120000080400036
:105830005e219000ee2190000288be000e0037002d
:10584000ce2190004e20900080004000008020007b
:1058500000804000100178007418b9000200400078
:10586000c200dd0000812000008040005e21900029
:10587000ee2190000288be000000eb0010079800a7
:105880001a0037004e2490004e2090008102200024
:105890008e8040004200dd00010040001002be008a
:1058a0004e2090001e0190007400b90002004000dc
:1058b000c200dd0000812000008040001001be0019
:1058c0000400be00d7eb07000001be0081022000eb
:1058d0008e8040004240dd00010040000288be0092
:1058e0001e0090000000e800100798004e20900075
:1058f0008000400000802000008040009000780080
:105900001e009000808f5000deff3d004e2590006d
:105910004e209000810220008e8040004200dd0079
:10592000010040001004be004e20900080004000a6
:105930000080200000804000100078000000e80097
:10594000cf80de008beb07000001be000800be0028
:1059500045ec07000001be00e80047004250dd00b2
:10596000010040000288be00ce209000018140006e
:105970000080200000004100100078000001e800d5
:1059800081804000008020000080400002087800f4
:105990004e209000e80047004200dd00010040007a
:1059a0001001be0022079800330798002e019000d6
:1059b000be0190004e209000040007004f057800c3
:1059c0004f04be000080fa00000006000a00fa0042
:1059d0002007980032079800430798006000b8003d
:1059e000008fbe0002002c00934724003e00900070
:1059f000ce0090005eec07000000e00001003200e5
:105a0000070037002e009000c200dd0000a9200032
:105a100000804000301f7800201778000700370012
:105a20002e009000c200dd0000a920000080400090
:105a30003e019000ce0190000288be001e00be0014
:105a40000080fa00000006000000fa002c03a80005
:105a50002c23a8002c43a8002c63a8002c83a800aa
:105a60002ca3a8002cc3a8002ce3a8002d03a80099
:105a70002d23a8002d43a8002d63a8002d83a80086
:105a8000c8a2a900c8c2a900c8e2a900c9e2a90029
:105a9000c902a900d002a900d022a900d042a900c1
:105aa000d062a900d0a2a900d0c2a900d0e2a9006a
:105ab000d102a900d122a900c002a800c022a800da
:105ac000c082a800c0e2a800c102a800c122a800ac
:105ad000c142a800c9a2a80069a0a900c9c2a80023
:105ae000c922a800d082a80000000000d4c2a800eb
:105af00000000000d4e2a80000000000d502a800c9
:105b000000000000d522a80000000000d402a80078
:105b100000000000d462a80000000000cde2a80050
:105b200000000000d4a2a80000000000cce2a80001
:105b300000000000d422a80000000000cca2a900b0
:105b400000000000ccc2a90000000000d442a9005f
:105b5000000000000000eb00a08f880000000000a3
:105b60000000eb00a08f8800000000000000eb00a8
:105b7000a08f88000080fa00000006000800fa00ec
:105b8000000f7800110798001e0090000000e00050
:105b900002003200100020001007980000000000f2
:105ba0001e0078006101b9002207980033079800b1
:105bb000f0002000010020002e019000be019000a6
:105bc000800f5100818f59009f003e002e009000f1
:105bd000be009000006001000f0037001900370080
:105be0002000370029003700330037003c00370021
:105bf000460037004d003700570037005e00370081
:105c000068003700720037007c00370086003700dc
:105c1000880037008a0037001e0090006140600055
:105c2000614060004601dd00412d20009140780078
:105c3000f0cbb30000c0600002407000d4e2b700b7
:105c4000810037001e00900061406000c700dd0049
:105c5000d4c2bf000074a10001407000d4e2b700bc
:105c6000790037001e0090006140600061416000d3
:105c7000512d200091407800e0cfb30000c06000bb
:105c800002407000d5e2b7006f0037001e009000a0
:105c9000614060006140600000414000512d2000e3
:105ca00091407800d0cfb30000c060000240700087
:105cb000d5e2b700640037001e009000614060002c
:105cc00061416000412d200091407800e0cfb30099
:105cd00000c0600002407000d4e2b7005a003700f4
:105ce0001e00900061406000614060004301dd00e3
:105cf000412d20009140780070cfb30000c06000bb
:105d000002407000d4e2b7004f0037001e00900040
:105d100061406000c700dd00cdc2bf000074a1007b
:105d200001407000cde2b700470037001e00900030
:105d300061406000614060004501dd00412d2000b0
:105d400091407800f0cdb30000c0600002407000c8
:105d5000d4e2b7003c0037001e00900061406000b4
:105d6000c700dd00ccc2bf000074a100014070007c
:105d7000cce2b700340037001e00900061406000a4
:105d80006140600000414000412d200091407800ba
:105d9000d0cfb30000c0600002407000d4e2b70072
:105da000290037001e0090006140600061406000e3
:105db0004501dd00c12c200091407800f0cdb300fa
:105dc00000c0600002407000cce2b7001e00370047
:105dd0001e00900061406000614060004601dd00ef
:105de000c12c200091407800f0cbb30000c06000cf
:105df00002407000cce2b700130037001e00900094
:105e000061406000614060004201dd00412d2000e2
:105e100091407800b0cfb30000c060000240700035
:105e2000d4e2b700080037009e009000a18f8800e0
:105e3000050037001e019000a28f88000200370085
:105e40009e019000a38f88000080fa0000000600e9
:105e50000800fa00000f7800000000000000eb00ce
:105e6000a08f88001e0078006101b9002207980009
:105e700033079800f0002000010020002e01900060
:105e8000be019000800f5100818f590070003e00cc
:105e90002e009000be009000006001000f0037004f
:105ea000150037001a0037001e00370024003700a5
:105eb000280037002e003700330037003900370044
:105ec0003e003700440037004a00370050003700da
:105ed00056003700580037005a003700d4c2bf00c0
:105ee0000080fb004600de00614060000080fb0097
:105ef0001007980058003700d4c2bf000080fb0094
:105f00004700de000080fb001007980052003700b9
:105f1000d5c2bf00614060000080fb001007980000
:105f20004d003700d5c2bf000080fb000000d1004b
:105f3000614060000080fb001007980046003700b9
:105f4000d4c2bf00614060000080fb0010079800d1
:105f500041003700d4c2bf000080fb004300de00d8
:105f6000614060000080fb00100798003a00370095
:105f7000cdc2bf000080fb004700de000080fb00b8
:105f80001007980034003700d4c2bf000080fb0027
:105f90004500de00614060000080fb0010079800b3
:105fa0002d003700ccc2bf000080fb004700de00a0
:105fb0000080fb001007980027003700d4c2bf0004
:105fc0000080fb000000d100614060000080fb0009
:105fd0001007980020003700ccc2bf000080fb00f3
:105fe0004500de00614060000080fb001007980063
:105ff00019003700ccc2bf000080fb004600de0065
:10600000614060000080fb0010079800120037001c
:10601000d4c2bf000080fb004200de00614060008f
:106020000080fb00100798000b003700a18f800054
:106030001107980008003700a28f8000120798000f
:1060400005003700a38f8000130798000200370077
:106050000000eb00100798001e0090000080fa007e
:10606000000006000600fa0020079800100020003b
:10607000000f78000000eb00100798000b003700bd
:106080002e0090001e006000800078001e0090002e
:10609000bafe07001e00780000004000000f7800e4
:1060a0001e0090000000e800100798001e009000fd
:1060b000ef0f5000f2ff34000080fa0000000600ed
:1060c0000600fa0010002000100798000000eb0006
:1060d000000f78000000eb00200798000c0037004c
:1060e0002e0090005aff07000000e000020032007e
:1060f0001e0090001e0f40001e0090000000400097
:10610000100798002e0090000000e800200798007b
:106110002e009000ef0f5000f1ff34001e007800b9
:106120000080fa00000006000800fa00000f780066
:10613000000000000000eb00a08f88001e00780027
:106140006101b9002207980033079800f000200091
:10615000010020002e019000be019000800f510030
:10616000818f590066003e002e009000be00900016
:10617000006001000f0037001300370019003700de
:106180001f00370025003700290037002f00370097
:10619000350037003a00370040003700460037002e
:1061a000480037004a0037004c0037004e003700e7
:1061b00050003700c3c2bf00614060000080fb0098
:1061c0001007980050003700c3c2bf000080fb00da
:1061d0000000d100614060000080fb0010079800c3
:1061e00049003700c3c2bf000080fb004200de0050
:1061f000614060000080fb001007980042003700fb
:10620000cbc2bf000080fb004500de0061406000a3
:106210000080fb00100798003b003700c2c2bf009f
:10622000614060000080fb001007980036003700d6
:10623000c2c2bf000080fb000000d10061406000ce
:106240000080fb00100798002f003700c2c2bf007b
:106250000080fb004400de00614060000080fb0025
:106260001007980028003700c2c2bf000080fb0062
:106270004700de000080fb00100798002200370076
:10628000cbc2bf000080fb004600de006140600022
:106290000080fb00100798001b003700d2c2bf002f
:1062a0000080fb004400de00614060000080fb00d5
:1062b0001007980014003700a18f80001107980084
:1062c00011003700a28f8000120798000e003700df
:1062d000a38f8000130798000b003700a08f800069
:1062e0001007980008003700a18f80001107980060
:1062f00005003700a28f80001207980002003700c7
:106300008001eb00130798001e0090000080fa0047
:10631000000006000600fa00100020001007980098
:106320000000eb00000f78000000eb002007980051
:106330000c0037002e0090007bff07000000e000fb
:10634000020032001e0090001e0f40001e00900050
:1063500000004000100798002e0090000000e800a8
:10636000200798002e009000ef0f5000f1ff34003e
:0c6370001e0078000080fa00000006000b
:020000040000fa
:10637c00761000008e0000000000000000080000f5
:10638c00f0020000000000000411000050000000aa
:10639c0002000000000000000000000000000000ef
:1063ac0000000000000000000000000000000000e1
:1063bc0000000000000000000000000000000000d1
:1063cc0000000000000000000000000000000000c1
:1063dc0000000000000000000000000000000000b1
:1063ec0000000000000000000000000000000000a1
:1063fc000000000000000000000000000000000091
:10640c00f01100000200000000000000f21100007a
:10641c000200000000000000ea110000060000006d
:10642c0000000000f4110000020000000000000059
:10643c00100d00005e01000000000000541100006f
:10644c00400000000000000094110000400000001b
:10645c0000000000d4110000160000000200000033
:10646c000000000000000000000000000000000020
:10647c00000000000000000000000100000000000f
:10648c006e0e00000801000000000000760f0000f6
:10649c00000100000200000029b30900285de000a3
:1064ac00185e27006e465500c48150000b7f2a00f1
:1064bc005708f30060ae99003dc0110014eb0700c3
:1064cc002fde3500d86570002c8b6d00e96c39001f
:1064dc00f0e5a000dbfb0f00ddf5ef0068b6210056
:1064ec008a3ba600f792be001f7dbc00726156006d
:1064fc009d6a03008e42450098b174003295f200fb
:10650c00901c1d005f25020075f64100b7cef1000e
:10651c00e6830d00913f6200c8b0e200059ebd000d
:10652c00311236001e78e30044305b0059fcd20077
:10653c00b9cb8c00ab9b3800a2f9c90086f44300a0
:10654c00c594f800526422005aec3300a7b2cf0075
:10655c00c1a4e100da934f0047d9970026c6d700b3
:10656c00d47b9c004c797100fd37ff001719e700b4
:10657c00bb154800d1675100230c06007a4e200051
:10658c003c5c0e00ca538000c387df00d3b55400b7
:10659c000077ad00a5ea2d00d06b8800c77e8d007a
:1065ac00a3b46300acdc4b0073e86f00e4cced00eb
:1065bc0049fe3e006984160024768f00a185a9004f
:1065cc000a34ba00b8aa4d00cd897c00ee109f00a9
:1065dc00fabf4a001b820400c2012e003a6640003a
:1065ec00a8965800d6afd5009a1a2b0000000000d0
:1065fc00f00a000020020000020000000000000071
:10660c00000000000000000000000000000000007e
:10661c00000000000000000000000000000000006e
:10662c00000000000000000000000000000000005e
:10663c00000000000000000000000000000000004e
:1068dc000000000020140000260000000200000050
:1068ec0022144800140000004814090000000000a5
:1068fc0002004600140000004614060002010000cd
:10690c000000000000000000000006000202000071
:10691c00000000004614000006000000000000000b
:10692c0056130000a000000002000000010000004f
:10693c000000000000000a00000000000000000041
:10694c00006400000000000000000000e8030000ec
:10695c0000000000000010002700000000000000f4
:10696c0000a08600010000000000000040420f0063
:10697c00000000000000800096980000000000005d
:10698c000000e100f50500000000000000ca9a00bc
:10699c003b00000000000000e40b5400020000006b
:1069ac000000e80076481700000000000010a50069
:1069bc00d4e8000000000000a0724e00180900008e
:1069cc00000040007a10f3005a0000000080c6005e
:1069dc00a47e8d000300000000c16f00f28623002e
:1069ec00000000008a5d780045630100000064002f
:1069fc00a7b3b600e00d000000e889000423c7002f
:106a0c008a000000f61300002a00000002000000bb
:106a1c00286e75006c6c2900003031003233340064
:106a2c0035363700383941004243440045460000b2
:106a3c00303132003334350036373800396162007a
:106a4c006364650066000000f61100006001000040
:106a5c00020000000000000000000000f03f0000f9
:106a6c000000a0009999b9003f0000000040e1002f
:106a7c007a843f0000000000e04d6200503f0000af
:106a8c000000e000e2361a003f0000000080b50074
:106a9c00f8e43e0000000000a0f7c600b03e000085
:106aac000000a000f2d77a003e00000000e08e004b
:106abc0079453e0000000000e00b2e00113e000066
:106acc000000e000df7cdb003d0000000000a100c6
:106adc009cc73b0000000000004c4800b43900008b
:106aec0000000000206ca100370000000000000036
:106afc00000000000000000000000000000000008a
:106b0c000000000000000000000000000000000079
:106b1c000000000000000000000000000000000069
:106b2c000000000000000000000000000000000059
:106b3c000000000000000000000000000000000049
:106b4c00000000000000f0003f000000000000000a
:106b5c00002440000000000000000000594000002c
:106b6c000000000000408f0040000000000000000a
:106b7c0088c340000000000000006a00f8400000dc
:106b8c000000000080842e00410000000000d000b6
:106b9c0012634100000000000084d7009741000000
:106bac000000000065cdcd004100000000205f001a
:106bbc00a002420000000000801daf001544000040
:106bcc0000004000593e2900460000000000000073
:106bdc0000f07f000000000000000000f07f0000cb
:106bec00000000000000f0007f000000000000002a
:106bfc0000f07f000000000000000000f07f0000ab
:106c0c00000000000000f0007f0000000000000009
:106c1c0000f07f000000000000000000f07f00008a
:106c2c00000000000000f0007f0000004c14000089
:106c3c000200000002000000010000000000000043
:020000040000fa
:106c4c000000fa0041d22000c0d220008008780059
:106c5c0041d220000000eb009000980041d22000af
:106c6c000000eb00a000980041d22000f0012000b1
:106c7c00b0009800012420009140780030ceb30081
:106c8c0000c060000024a00040e2b7004342a8000e
:106c9c0042e2a80042a2a9002124200091407800e1
:106cac0030ceb30000c060008041b30042e2b700b8
:106cbc0042c2bf003040b30042e2b7004402a90018
:106ccc0040c2a90041e2a8008540a900a9c0bf00ac
:106cdc007040b300a9e0b7009540a8000080fa000e
:106cec00000006000400fa001007980009090700cc
:106cfc0041d220001e0090000a030700000f78000c
:106d0c000e0907001e0078000080fa000000060043
:106d1c000000fa00d06880000080fa000000060035
:106d2c000000fa00e06880000080fa000000060015
:106d3c000000fa00006980000080fa0000000600e4
:106d4c000000fa00f06880000080fa0000000600e5
:106d5c000000fa00106980000080fa0000000600b4
:106d6c000000fa00906880000080fa000000060025
:106d7c000000fa000000eb00d06888000080fa00e8
:106d8c00000006000000fa000000eb00e06888003c
:106d9c000080fa00000006000000fa000000eb0082
:106dac00006988000080fa00000006000000fa006c
:106dbc000000eb00f06888000080fa00000006007c
:106dcc000000fa000000eb00106988000080fa0057
:106ddc00000006000000fa000000eb00906888003c
:106dec000080fa00000006000601fa0080688000ae
:106dfc000000e0002c0032006600470021e2290070
:106e0c00ff000900315878000010b1000000eb00c1
:106e1c0010079800090037001e0190002e0090000a
:106e2c00804078006600470000004100014878006f
:106e3c001e0090000000e800100798006400470056
:106e4c0041d22000b70207000000e000f2ff3a0038
:106e5c0040d22000d6020700c0d62000021020002d
:106e6c008000eb00cbeb07006600470021f2290005
:106e7c0051040700000f78001e00780010407800c5
:106e8c000004e000040032004200200061f52900fb
:106e9c001e0078009d0407000000eb00906888003d
:106eac000000eb00806888000080fa0000000600fb
:106ebc00809fbe000800fa00cc82a800401280001f
:106ecc0020079800ae00900061738800d0688000a5
:106edc000000e800d0688800b06880000000e00086
:106eec0087003a002e0090004a00de001007980040
:106efc00ae009000f03f2000008f60001e00780074
:106f0c00c06888009e009000310798003e009000f9
:106f1c00e40f50003b003200be009000e48f5000a4
:106f2c000a003e003e009000e20f500023003200a9
:106f3c00be009000e28f50002f003e003e009000fb
:106f4c00e10f50000b0032004d003700be009000e6
:106f5c00e68f5000330032003e009000e60f5000e8
:106f6c002c003900be009000e78f50003e0032002c
:106f7c004300370010002000b0688800701020001b
:106f8c009e0f10000a003e00c06880008000780050
:106f9c00e0e6200000804000104078008080fb007c
:106fac000040200000804000401288007b00370029
:106fbc000000eb0040128800780037002000200011
:106fcc00b0688800f00f20009e0f100007003e00f4
:106fdc00c06880008000400000af200000804000ae
:106fec0010007800401288006c0037000000eb00a5
:106ffc00401288006900370030002000b06888001b
:10700c0066003700e06880000000e800e068880057
:10701c0062003700e06880000000e800e06888004b
:10702c005e003700806880000000e0000b003a0032
:10703c00c1688000f00f2000808f500007003e00d8
:10704c00c1688000c0d6200000804000104078004d
:10705c000000fb0040128800500037000000eb00dd
:10706c00401288004d003700f03f20009e0f1000aa
:10707c0003003a00100020008068880047003700a9
:10708c00e06880000000e800e068880040d2200042
:10709c00100090008000e80040d2200030009000ea
:1070ac008080600040d2200020009000808f500033
:1070bc0003003a0010002000906888003700370069
:1070cc0040d220009000780040d2200010009000a8
:1070dc0000004000008040001e08780040d22000d4
:1070ec00100090008000e80040d22000300090009a
:1070fc008080600040d220001100980027003700eb
:10710c00b0688000e10f500006003a000069800072
:10711c000000e800006988000000eb00b0688800ff
:10712c001e003700b0688000e20f500006003a00e5
:10713c00f06880000000e800f06888000000eb00b8
:10714c00b068880015003700b0688000e30f50006d
:10715c0010003a00c1688000f00f2000808f5000b2
:10716c0006003e00c06880008000400000af200098
:10717c0000804000ae00900001087800106980008b
:10718c000000e800106988000000eb00b06888007f
:10719c00020037000000eb00b0688800cc82a90028
:1071ac008540a9000080fa004f00be000040060098
:1071bc000200fa000000eb00000f780027003700f7
:1071cc009e0178001e0078004700dd0080007800ea
:1071dc00200821000080400000017800a107210058
:1071ec004318dd0001004000020878001e00780002
:1071fc00a10721004300dd000080e8008100400071
:10720c000000eb00800878001e007800a107210028
:10721c004300dd0064004000810040000000eb00f2
:10722c00800878001e007800a10721004300dd00d3
:10723c006600400081004000f007200080087800c4
:10724c001e0078008000400020102100808040004b
:10725c000000eb00800878001e0fe8001e00e00024
:10726c00d7ff3400b00020004011880021e2a800b4
:10727c0020a2a9002062a900004020001011880063
:10728c008560a9008580a900910a200091407800b2
:10729c00f0c8b30000c0600001c6b300014070002c
:1072ac00a9e0b700a10a20009140780080cfb3007c
:1072bc0000c060000014a000aae0b7009560a80010
:1072cc009580a9000080fa00000006000800fa0072
:1072dc0010079800210798001e009000e10f500045
:1072ec00010032000e0037008a0707001e009000d4
:1072fc004300dd0080007800a007210068005000ea
:10730c00808040002e0090000a010700000f7800da
:10731c008a0707001e007800300798000500370028
:10732c00ae0090000040eb00804878000000eb00bd
:10733c00300798003e0090000080fa000000060024
:10734c000800fa0010079800414798001e009000b2
:10735c00e10f5000010032000700370023c2bf00cc
:10736c000080fb000000d100614060000080fb0049
:10737c00000f78000200370010002000000f78008a
:10738c001e00e0000a003a001e009000e10f5000c1
:10739c0001003200060037004e4090000080fb00d8
:1073ac0020118800100020003007980002003700e0
:1073bc000000eb00300798003e0090000080fa00bf
:1073cc00000006000600fa0010079800210798003c
:1073dc000000eb00000f78000b0037001e00780057
:1073ec00800078002e009000008040001040780053
:1073fc00804078001e009000d1ff07000000e000e4
:10740c00010032001e0fe8001e007800800078009a
:10741c002e00900000804000104078000004e00036
:10742c00eeff3a000000eb000080fa0000000600be
:10743c000600fa00100798001e009000e10f5000a3
:10744c00010032000d003700320707001e009000cb
:10745c004300dd0080007800a00721006800500088
:10746c0000804000e1000700000f780033070700a0
:10747c001e00780020079800020037000000eb0087
:10748c00200798002e0090000080fa0000000600f3
:10749c000400fa00100798001e009000e10f500045
:1074ac00010032000700370023c2bf000080fb0040
:1074bc000000d100614060000080fb00000f7800ec
:1074cc000200370010002000000f78001e0078002a
:1074dc000080fa00000006000400fa00000f78009b
:1074ec001e007800e10f5000010032000700370049
:1074fc001e00780080004000201021000080400019
:10750c001000780010079800020037000000eb0014
:10751c00100798001e0090000080fa000000060082
:10752c000200fa00000f78001e007800e10f5000f6
:10753c0001003200060037001e0078008000400079
:10754c0020102100808040000000eb0080087800b3
:10755c000080fa00000006000400fa0010079800f2
:10756c001e009000e10f50000100320013003700a4
:10757c00e80607001e0090004300dd008000780044
:10758c00a007210068005000008040008d0007001b
:10759c001e009000e10f500003003200060037007f
:1075ac0030118000000f780022c2bf0061406000e3
:1075bc000004e000faff3a00e00607000080fa0041
:1075cc00000006000200fa00000f78001e00780090
:1075dc00e10f500001003200040037002342a900e3
:1075ec00000000002342a800000000000080fa0008
:1075fc0000000600809fbe000000fa00b0838000ef
:10760c00c183800061004000e0804800b0838800a6
:10761c00c18388008580a9000080fa004f00be005d
:10762c0000400600809fbe000000fa001c003700de
:10763c00a0072100100090008000e800a0072100a6
:10764c003000900080806000a00721002000900096
:10765c00808f500003003a00100020001088880032
:10766c000f003700a007210090007800a007210030
:10767c00100090008080400030118000804878001d
:10768c00a0072100100090008000e800a007210056
:10769c003000900080806000a0072100110098004d
:1076ac0022c2bf00614060000004e000e0ff3a002d
:1076bc008560a9000080fa004f00be000040060063
:1076cc000600fa00004f7800110798001e00900089
:1076dc00460007000000e000030032000000eb0051
:1076ec0020079800100037001e00900090007800d2
:1076fc001e00900010009000008040001e48780092
:10770c001e009000100090008000e8001e00900009
:10771c0030009000808060001e00900011009800e6
:10772c0010002000200798002e0090000080fa0026
:10773c00000006000600fa00000f78001107980000
:10774c001e0090003d0007000000e0000600320023
:10775c009e0078000040eb00804878000000eb00b1
:10776c00200798001400370060172a007fe90700f3
:10777c001e009000900078001e00900020009000e9
:10778c0000804000904078001e007800014878008e
:10779c001e009000200090008000e8001e00900069
:1077ac0030009000808060001e0090002100980046
:1077bc0010002000200798002e0090000080fa0096
:1077cc00000006000200fa00000f78009e0078000e
:1077dc000000eb00a00098009e0078000000eb0079
:1077ec00900098000080fa00000006000400fa00e7
:1077fc00000f78001e007800100090008000e80058
:10780c001e00780030009000808060001e00780020
:10781c0020009000808f500003003a0010002000e0
:10782c0010079800020037000000eb0010079800ca
:10783c001e0090000080fa00000006000400fa0010
:10784c00000f78001e007800a00090001e00780049
:10785c0010009000808f500003003a0010002000b0
:10786c0010079800020037000000eb00100798008a
:10787c001e0090000080fa00000006000200fa00d2
:10788c00000f78001e007800900090001e00780019
:10789c0020009000808050001e0078003000900086
:1078ac00008060000080fa00000006000600fa006c
:1078bc00000f7800110798001e009000460007008a
:1078cc000000e000030032000000eb0020079800ed
:1078dc00110037001e009000900078001e009000f0
:1078ec001000900000004000008040001e0878004e
:1078fc001e009000100090008000e8001e00900018
:10790c0030009000808060001e00900011009800f4
:10791c0010002000200798002e0090000080fa0034
:10792c00000006000600fa00000f7800110798000e
:10793c001e0090003c0007000000e0000600320032
:10794c009e0078000000eb00800878000000eb003f
:10795c0020079800130037001e009000900078005c
:10796c001e009000200090000000400000804000ad
:10797c00900078001e007800010878001e0090002e
:10798c00200090008000e8001e0090003000900065
:10799c00808060001e0090002100980010002000e4
:1079ac00200798002e0090000080fa0000000600ce
:1079bc000200fa00000f78009e0078000000eb0037
:1079cc00a00098009e0078000000eb00900098004a
:1079dc000080fa00000006000400fa00000f780096
:1079ec001e007800100090008000e8001e00780057
:1079fc0030009000808060001e0078002000900015
:107a0c00808f500003003a001000200010079800ef
:107a1c00020037000000eb00100798001e009000d9
:107a2c000080fa00000006000400fa00000f780045
:107a3c001e007800a00090001e007800100090003e
:107a4c00808f500003003a001000200010079800af
:107a5c00020037000000eb00100798001e00900099
:107a6c000080fa00000006000200fa00000f780007
:107a7c001e007800900090001e00780020009000fe
:107a8c00808050001e007800300090000080600064
:107a9c000080fa00000006004800fa00201f980041
:107aac00311f9800421f98006400470061142a009f
:107abc0017000900311878000003b1004e1990002e
:107acc0032279800be219000e18f51004300320014
:107adc003e209000e20f50007c003200be2090004f
:107aec000100e00001003200b400370064014700df
:107afc000000200001f823000089be00640147004b
:107b0c000000200001f823002001980031019800aa
:107b1c00640147000000200001f823004001980098
:107b2c0051019800640147000000200001f8230077
:107b3c00600198007101980064014700000020006a
:107b4c0001f823000009980011099800640147000e
:107b5c000000200001f8230020099800310998004a
:107b6c00640147000000200001f823004009980040
:107b7c0051099800640147000000200001f823001f
:107b8c00600998007109980064014700000020000a
:107b9c0001f82300001198001111980064014700ae
:107bac000000200001f823002011980031119800ea
:107bbc00640147000000200001f8230040119800e8
:107bcc0051119800640147000000200001f82300c7
:107bdc0060119800711198007d0037006401470016
:107bec0080002000018223000089be006401470050
:107bfc0080002000018223002001980031019800b0
:107c0c00640147008000200001822300400198009d
:107c1c00510198006401470080002000018223007c
:107c2c0060019800710198006401470080002000f9
:107c3c000182230000099800110998006401470093
:107c4c00800020000182230020099800310998004f
:107c5c006401470080002000018223004009980045
:107c6c005109980064014700800020000182230024
:107c7c006009980071099800640147008000200099
:107c8c000182230000119800111198006401470033
:107c9c0080002000018223002011980031119800ef
:107cac0064014700800020000182230040119800ed
:107cbc0051119800640147008000200001822300cc
:107ccc006011980071119800410037006401470061
:107cdc00a000200081ac23000089be006401470095
:107cec00a000200081ac23002001980031019800f5
:107cfc0064014700a000200081ac230040019800e3
:107d0c005101980064014700a000200081ac2300c1
:107d1c00600198007101980064014700a0002000e8
:107d2c0081ac2300000998001109980064014700f8
:107d3c00a000200081a4230020099800310998009c
:107d4c0064014700a000200081ac2300400998008a
:107d5c005109980064014700800020000182230033
:107d6c0060099800710998006401470070002000b8
:107d7c00017823000011980011119800640147004c
:107d8c007000200001782300201198003111980018
:107d9c006401470070002000017823004011980016
:107dac0051119800640147008000200001822300db
:107dbc006011980071119800050037000200200036
:107dcc0003f82b0012279800232798001f00370078
:107ddc002e189000e40047004200dd000100400036
:107dec001001be00721f9800032798003e189000e7
:107dfc00cf80de005ce20700501f9800611f9800e6
:107e0c003e1890000000e00007003d00020020003a
:107e1c00037824005e189000ee1890007ee20700b4
:107e2c00501f9800611f98005e199000ee19900089
:107e3c007e1890008e209000d4e20700008fbe00c8
:107e4c001e00be0010279800212798001e209000cd
:107e5c00ae2090000080fa00000006000800fa0036
:107e6c00881f780010079800210798000000eb008d
:107e7c00000f78001e009000104078000004e00015
:107e8c0003003a000000eb00300798004600370072
:107e9c001e007800800078002e00900000804000ca
:107eac00104078000000fb00c2e1070000047800dd
:107ebc001e007800800078001e00900000804000ba
:107ecc00104078000000fb00bae10700800f54005e
:107edc00150032002e0090000000e80020079800ea
:107eec002e009000104078000004e00003003a00df
:107efc000000eb00300798002b0037002e0090009c
:107f0c0090407800c0c7b30080cf5000f1ff3a001a
:107f1c002e0090000000e800200798000000eb0005
:107f2c00000f78001b0037001e0fe8001e007800c1
:107f3c00800078002e0090000080400010407800f7
:107f4c000004e000080032001e0078008000780079
:107f5c002e0090000080400090407800c0c7b30015
:107f6c0080cf50000b003a001e0078008000780093
:107f7c001e00900000804000104078005200070066
:107f8c000000e00003003a001e0078003007980063
:107f9c0005003700700220009e0f1000bcff34005b
:107fac001e007800300798003e0090004f047800c7
:107fbc000080fa00000006000600fa001007980086
:107fcc00210798000080eb00000f78000e003700ae
:107fdc001e009000104178001e0078008000780090
:107fec002e0090000080400010407800804f51001f
:107ffc0005003a001e0090000000e80010079800f1
:10800c000080eb00000f78001e0fe8001e007800c7
:10801c00800078002e009000008040001040780016
:10802c000004e000eaff3a001e0090000080fa0015
:10803c00000006000400fa00000f780081182a00e6
:10804c001e007800dcff0700000f78001e0078008f
:10805c0090407800d0c2b30080cf500005003200b1
:10806c001e00780090407800b0c2b30080cf500062
:10807c0001003a001e0fe800b1182a001e0078001b
:10808c00cdff0700000f7800d1182a001e007800e1
:10809c00c9ff0700000f78001e0078001040780020
:1080ac000004e000030032000000eb001007980011
:1080bc000200370010002000100798001e009000ee
:1080cc000080fa00000006000400fa00004f78005f
:1080dc001e00fb003ee107000000e00003003a0038
:1080ec00f0c5b3009e4f100003003a0010002000b2
:1080fc0010079800020037000000eb0010079800f2
:10810c001e0090000080fa00000006000c00fa002f
:10811c002007980031079800420798000000eb00f8
:10812c00000f780081182a002e009000a2ff070093
:10813c00200798001e0037001e0078004200dd006a
:10814c00800078003e009000008040009000780095
:10815c002e00900041ff0700100798001e009000b1
:10816c000000e000110032001e009000800078003a
:10817c002e0090000080400081182a008eff07001e
:10818c00200798001e0078004200dd008000780077
:10819c003e00900000804000900090002e00900067
:1081ac0001000100500798000c0037001e0fe8007a
:1081bc001e0078004200dd00800078003e00900038
:1081cc000080400010007800104078000004e000af
:1081dc00d9ff3a004e009000500798005e009000c6
:1081ec000080fa00000006000000fa000000eb001e
:1081fc00800888000000eb0030088800f07f240025
:10820c006008880084e0a90094e0a80011e1a800af
:10821c000080fa00000006000000fa00b30007001e
:10822c000080fa00000006000200fa00000f78003f
:10823c001e007800100078000080fa000000060094
:10824c000200fa00000f78001e007800640007009e
:10825c001e007800020007000080fa0000000600f3
:10826c000200fa00000f78001e0178006000b800d0
:10827c003001980041019800960007001e0178001b
:10828c0010019800210198000080fa0000000600ff
:10829c000600fa00200798008e000700008fbe0031
:1082ac002e009000100078000000e0002300320047
:1082bc002e009000a000900010009000be0f500007
:1082cc00ae8f58000f0036002e0090003001900049
:1082dc00c00190002e009000a000900010009000b3
:1082ec003e024000ae8248000400be000200400086
:1082fc00838048002e0190003001980041019800c5
:10830c000e0037002e00900030019000c00190004c
:10831c002e009000a0009000100090003e02100073
:10832c00ae8218000400be000200400083804800aa
:10833c002e01900030019800410198002e00900011
:10834c001e01be0012009800230098002e00900021
:10835c0030039000c003900086007800a00020003d
:10836c00000ab8006030b900050178000001410036
:10837c006a38b90000014100820278000400be0096
:10838c000080fa00000006000200fa00000f7800de
:10839c001e007800beff07009e0078001000200031
:1083ac00800878001e00780030039000c003900015
:1083bc0086007800a0002000000ab8006030b900e8
:1083cc0005017800000141006a38b9000001410044
:1083dc00820278000400be000080fa000000060053
:1083ec000200fa00000f78001e007800a8ff0700ba
:1083fc009e0078000000eb00800878001e007800da
:10840c0030039000c003900086007800a00020008c
:10841c00000ab8006030b900050178000001410085
:10842c006a38b90000014100820278000400be00e5
:10843c000080fa00000006000600fa0020079800f1
:10844c00240007000001be002e0090000100200057
:10845c00001f4100019749001e000700be0f50008d
:10846c00ae8f5800fcff39000080fa0000000600b7
:10847c000600fa002007980016000700008fbe00c7
:10848c002e009000e90f5000080036002e009000de
:10849c00a2002000110009000280d8000100200079
:1084ac001e0f40005e9748000400370010002000ab
:1084bc00010020001e0f40005e97480005000700d9
:1084cc00be0f5000ae8f5800fcff39000080fa0040
:1084dc00000006000000fa0004000700608f800016
:1084ec00718f80000080fa00000006000200fa0084
:1084fc00528f8000608f8000718f8000000f5100c0
:10850c001e0078006101b800608f8000718f8000c0
:10851c000200400083804800608f8800718f8800c3
:10852c000080fa0000000600801f78000000fa00ae
:10853c000000eb0030088800508f80000000e8003d
:10854c00508f880084e0a9000080fa004f0078006a
:10855c00004006008c00fa000000eb00000f7800d1
:10856c00416a20009140780000ceb30000c060004a
:10857c009040b300a4e6b700816c200091407800d5
:10858c0000ceb30000c060003040b300c8e6b700b6
:10859c00c8e2a900cce2a800b16c200091407800a0
:1085ac0000ceb30000c060007040b300cbe6b70053
:1085bc00816a20009140780000ceb30000c06000ba
:1085cc00a040b300a8e6b700916a20009140780063
:1085dc0000ceb30000c06000c040b300a9e6b700f5
:1085ec00a16a20009140780000ceb30000c060006a
:1085fc00d040b300aae6b70010f50700ecfa07006c
:10860c00f9fe07008ef907001e0207005001070053
:10861c0080002000e3f2070070c8b3005c02070082
:10862c0030062000dff2070090002000ddf207008a
:10863c0070c8b3005602070030062000d9f20700bc
:10864c00e8004700e0082a00801f780070092a0023
:10865c00801f7800300a2a00801f78000100780003
:10866c00f8e50700e6875700e800470010002000f7
:10867c0054fb0700800720000e004000f8fe0700a6
:10868c00800720000e0040003fff0700200820005c
:10869c000e004000f2fe0700200820000e004000f3
:1086ac0039ff070068004700300007000000e000b9
:1086bc0003003a003000200030079800100037000b
:1086cc0068004700a10d2a003bfe07002007980018
:1086dc002e009000104078000004e00003003a00e7
:1086ec0020002000300798000500370042002000d1
:1086fc0061f529002e00900084fe070030079800d9
:10870c003e009000e30f5000150032003e00900038
:10871c000000e0000f0032003e009000e20f50001d
:10872c000c003200800520000e004000be009000be
:10873c00811f7800010e2a00811f7800c1e5070017
:10874c00e4875700810520008e8040001000200037
:10875c001cfb0700b10e2a001000200019fb0700bb
:10876c003d010700a0f90700ceff37000800fa0012
:10877c00300798000000eb0010079800e400470059
:10878c0010002000d1fa07000000e0003f0032008a
:10879c00ce40900010002000e9fa07004e409000f7
:1087ac00ed4f500003003a00a1c0b30010002000b0
:1087bc00e3fa07004e409000ed4f50001a003200d3
:1087cc004e409000e84f50000d003200818f800029
:1087dc00f0042000808f500009003c00828f800044
:1087ec004e40900080407800401021000000410075
:1087fc00014878000200e800808f880006003700ee
:10880c00808f80000000e00003003400808f800027
:10881c000000e900808f8800be0090000040eb0053
:10882c0080487800190037001000200010079800cd
:10883c00818f800040102100808040000040eb00c0
:10884c00804878000000eb00000f78000a00370029
:10885c001e007800800078003e00900000814000ef
:10886c009e007800401021000080400010407800ed
:10887c00004978001e0fe800808f80009e0f1000ca
:10888c00f3ff34000000eb00808f88001e00900086
:10889c000080fa00000006000a00fa001007980099
:1088ac0041479800320798001e0090000000e0003d
:1088bc00030032003e0090000000e00003003a008c
:1088cc001000200040079800340037001e00900074
:1088dc0037e50700000f78009e80e800f00f2000bd
:1088ec00808f5000030036001000200040079800d5
:1088fc002a0037003e009000e70040003e00900048
:10890c00704092000080fb00008040009e009000b0
:10891c002de507003e009000f04092001e0078000c
:10892c0080c040003e00900071409a003e009000d4
:10893c00e70040003e009000704092000080fb0079
:10894c00808040000040eb00804878003e009000a2
:10895c00704092008040e8003e00900071409a0008
:10896c003e009000e70040003e00900070409200f6
:10897c000080fb00808040004e40900080487800d2
:10898c003e009000704092008040e8003e00900055
:10899c0071409a000000eb00400798004e009000d8
:1089ac000080fa00000006001c00fa00400f98003e
:1089bc000000eb00200798004e0890000000e0003b
:1089cc00610032004e089000104078000080fb00df
:1089dc00801f7800200f2a00801f7800401921008a
:1089ec0018e50700e487570041192100100020000a
:1089fc0074fa07004e0890000000e800801f780011
:108a0c0020102a00801f7800401921000de5070076
:108a1c00e4875700411921001000200069fa070073
:108a2c0021112a001000200066fa07000000eb005c
:108a3c00300798003e0037004e089000e7004000d9
:108a4c002e0090008080400068004700020120004a
:108a5c00e5e4070091c0b3001000200038fa0700cd
:108a6c00e80047001000200056fa07006800470095
:108a7c00cfe40700800078002e0090000100400039
:108a8c00200798002e0090000000e80020079800b6
:108a9c002e009000ce0890006600400001004000bf
:108aac00104090000000fb00100798002e00900072
:108abc000000e800200798001e009000500f98005e
:108acc005e089000e20f50000b0032005e08900030
:108adc00e30f50000c0032005e089000e10f5000d4
:108aec00010032000c00370041122a001000200057
:108afc0034fa07000b003700e1122a0010002000a6
:108b0c0030fa07000700370091132a0010002000ec
:108b1c002cfa07000300370031142a001000200043
:108b2c0028fa07003e0090000000e800300798008b
:108b3c004e089000604090008080fb003e0090004a
:108b4c00808f5000bcff3e000080fa000000060041
:108b5c002600fa00881f78000e80e800e1052a0044
:108b6c0011000900311878004002b10050c0b30068
:108b7c006eeeb700f0e6200021082a000400090080
:108b8c003158780020c1b30074eeb700e2e6200043
:108b9c0011c0b30070082a003fff070061002000dd
:108bac0070082a003f01070012c0b3008000eb00e0
:108bbc005f0007000000eb00000f7800200037007a
:108bcc001e0078008e80e800000040006080780075
:108bdc00e2e620008040eb002fff07001e04780027
:108bec001e0078008e80e800000040006080780055
:108bfc006fe40700000178001e0078008e80e8000a
:108c0c000000400060807800820078002501070099
:108c1c0080407800401d210000004400014878008d
:108c2c009e007800401d210000804000104078001c
:108c3c000041eb009e0078003d0007001e0fe8008d
:108c4c00000120009e0f1000ddff36004f0478005d
:108c5c000080fa00000006000200fa00881f78006d
:108c6c00318f8000408f8000008f4000408f80004b
:108c7c00308f88001e007800408f88004100200053
:108c8c0080002a00070107000041eb009e007800dd
:108c9c00270007004000200020f5070000047800a2
:108cac005100200050042a00fe0007000041eb0098
:108cbc00880078001e0007005000200017f5070000
:108ccc000004780051002000b0042a00f5000700d1
:108cdc000041eb00880078001500070060002000c0
:108cec000ef50700000478005100200010052a0042
:108cfc00ec0007000041eb00880078000c00070036
:108d0c007000200005f507000004780051002000d9
:108d1c0070052a00e30007000041eb008800780092
:108d2c00030007004f0478000080fa0000000600e2
:108d3c000a00fa004047980031079800024f98004b
:108d4c004e4090000080fb004300de000080fb00e2
:108d5c00100798004e4090008080fb001e00900091
:108d6c004300dd0000805000670f10004e40900063
:108d7c000080fb008000400000af2000008040001d
:108d8c00be009000010878000e4890000080fb00a7
:108d9c0060004000e10f50000f003e009e0190006b
:108dac009e00900000cf2000008040001040780012
:108dbc00004178000e4890008080fb001e00780077
:108dcc000008dd00004069008040780000cf2000e2
:108ddc0000804100014878000080fa000000060085
:108dec000a00fa00404798003107980042079800a3
:108dfc004e4090000080fb004300de000080fb0032
:108e0c00100798004e4090008080fb001e009000e0
:108e1c004300dd0000805000670f10003e00900002
:108e2c000000e000080032004e4090000080fb0083
:108e3c008000400000af20000080400090007800cf
:108e4c003e009000010878004e0090000000e00009
:108e5c000a0032009e00900000cf200000804000ed
:108e6c00104078008080fb001e0078000088de0037
:108e7c00e14060004e009000014878000080fa004c
:108e8c00000006000000fa006382a9006362a900da
:108e9c006342a9006322a9006302a90062e2a9004f
:108eac0062c2a90062a2a80021262000914078008d
:108ebc0030ceb30000c0600062e2b70062c2bf00f7
:108ecc003040b30062e2b70065e2a90065c2a900b8
:108edc0065a2a9006422a9006402a90061e2a800ad
:108eec00811f7800821f7800831f78002174200076
:108efc0062042000730520008248780083487800c3
:108f0c0042c7a900cf0178004f017800cf0078004c
:108f1c00c16a20009140780000ceb30000c0600010
:108f2c000014a000ace6b700316c20009140780032
:108f3c0000ceb30000c06000a040b300c3e6b70091
:108f4c00416c20009140780000ceb30000c060005e
:108f5c00b040b300c4e6b700811f7800821f7800d0
:108f6c00831f780021742000620420007305200008
:108f7c00824878008348780042c7a800cf01780067
:108f8c004f017800cf0078000080fa000000060046
:108f9c000200fa00004f78001e80fb00401388008e
:108fac0060c2bf00614060000004e000fcff3200c2
:108fbc000040eb00004f7800401380000080fa0066
:108fcc00000006001800fa00100f98006000b800ae
:108fdc0070079800010f98000000eb0060079800e4
:108fec001e089000e70f5000050036007e00900030
:108ffc008e089000200f9800310f98002500370044
:10900c00ee0090006008200000807000600798005f
:10901c001e089000c600dd006e009000010070007c
:10902c006007980060c2a800000000006e0090006d
:10903c00d7ff0700000000000040eb00d4ff070042
:10904c00500798000040eb00d1ff07004007980044
:10905c000040eb00ceff070030079800de009000c8
:10906c00210798002e0090004800dd002007980092
:10907c00ce009000f00f2000808060002e00900049
:10908c0001007000200798006000b800200f9800c5
:10909c00310f98002e089000be0890000080fa0056
:1090ac00000006000800fa0020079800310798001d
:1090bc000040eb00204798000000eb00000f780008
:1090cc000d0037002e4090000081fb009e007800c0
:1090dc002e00900000804000104078000000fb0043
:1090ec008000690060f7200000804000904078000c
:1090fc00214798001e0fe8003e0090009e0f1000c4
:10910c00f0ff39002e4090000080fb000080fa0038
:10911c00000006000000fa00908f80000000e000c4
:10912c0001003a00ff3ffc00908f80000000e80037
:10913c00908f88000080fa00000006000000fa0002
:10914c00908f80000000e900908f8800908f800045
:10915c000000e00001003a000000fc000080fa0072
:04916c0000000600f9
:00000001FF
